:100000000C9491020C94AE020C94AE020C94AE02CD
:100010000C94AE020C94AE020C94AE020C94AE02A0
:100020000C94AE020C94FD120C94AE020C94AE0231
:100030000C94D7220C94AE020C94AE020C94AE0237
:100040000C94AE020C94AE020C94AF110C94AE0260
:100050000C94BE060C94AE020C9486060C94AE0270
:100060000C94FF150C94AE020C94E4210C94AE0297
:100070000C94E2520C94AE020C94AE0270197C19EE
:1000800011181D1837183216E017F2172D175D16C4
:100090003216511862187C189C18BC1816194E1686
:1000A00065227B2251229522702209229C2236222F
:1000B00023226C22602227222B22232291228C22AF
:1000C00027222B22232288225B22272246220A0A69
:1000D0000D004E65757472616C0048656164696EEF
:1000E00067486F6C64000A0D537465756572756EB0
:1000F000673A20004F4B0A0D000A0D4162676C659C
:10010000696368204C756674647275636B73656EA1
:10011000736F722E2E000A0D42656E75747A65201B
:10012000506172616D657465727361747A202564C3
:10013000000A0D414343206E696368742061626761
:1001400065676C696368656E21003A2047656E6576
:10015000726174696E672044656661756C742D50B8
:100160006172616D65746572207573696E67206F69
:100170006C6420537469636B2053657474696E6793
:1001800073000A0D496E69742E20454550524F4D3B
:10019000000A0D3D3D3D3D3D3D3D3D3D3D3D3D3D2F
:1001A0003D3D3D3D3D3D3D3D3D3D3D3D3D3D3D3D7F
:1001B0003D000A0D466C69676874436F6E74726F18
:1001C0006C0A0D48617264776172653A25642E2568
:1001D000640A0D536F6674776172653A5625642E12
:1001E0002564256320002E0048693A2534692020C3
:1001F00043663A253469200047733A253469202044
:1002000047693A25346920004E693A25346920202F
:10021000526F3A253469200045787465726E436FD9
:100220006E74726F6C20200052616E67653A2533E0
:10023000692D253369005374656C6C756E673A20BF
:1002400025336900536574706F696E7420202533FF
:100250006900536572766F202000506F7469343ADC
:10026000202025336900506F7469333A20202533EC
:100270006900506F7469323A202025336900506F4D
:100280007469313A20202533690053746172743ADD
:100290002020202020253569004D65737377657215
:1002A000743A2020253569005269636874756E6759
:1002B0003A2020253569004B6F6D706173732020E3
:1002C000202020202000456D70662E506567656CEB
:1002D0003A253569005370616E6E756E673A20205D
:1002E00025356900486F6368202534692028253347
:1002F000692900526F6C6C202534692028253369E8
:1003000029004E69636B202534692028253369292B
:1003100000414343202D2053656E736F720047697F
:1003200065722025346920282533692928253369F9
:100330002900526F6C6C20253469202825336929E7
:100340002825336929004E69636B202534692028EC
:1003500025336929282533692900476965722025D5
:10036000346920282533692900526F6C6C202534AC
:100370006920282533692E257829004E69636B2072
:1003800025346920282533692E2578290047696599
:10039000722025346920282533692900526F6C6C3E
:1003A0002025346920282533692E256929004E69C6
:1003B000636B2025346920282533692E256929009F
:1003C0004779726F202D2053656E736F7200503322
:1003D0003A253469202050343A25346920005031C0
:1003E0003A253469202050323A2534692000477379
:1003F0003A253469202047693A25346920004E693E
:100400003A2534692020526F3A25346920004B3751
:100410003A25346920204B383A25346920004B3581
:100420003A25346920204B363A25346920004B3375
:100430003A25346920204B343A25346920004B3169
:100440003A25346920204B323A25346920004B6F1D
:100450006D706173733A20202025356900526F6CEE
:100460006C3A202020202020253569004E69636BDE
:100470003A20202020202025356900616B742E2031
:100480004C6167650048F668656E726567656C75F6
:100490006E67004B65696E6520004F666620202000
:1004A0002020203A20253569004C756674647275E9
:1004B000636B3A2025356900536F6C6C486F656833
:1004C000653A2025356900486F6568653A20202027
:1004D00020202535690028632920486F6C676572E4
:1004E00020427573730053657474696E673A2025F2
:1004F00064200048573A5625642E25642053573A05
:1005000025642E25642563002B204D696B726F4B8B
:100510006F70746572202B005B25695D005B256937
:100520005D0011241FBECFEFD0E1DEBFCDBF13E0D1
:10053000A0E0B1E0EAEDFCEA02C005900D92A23C19
:10054000B107D9F718E0A2ECB3E001C01D92AB3EB1
:10055000B107E1F70E9459030C946C560C9400000B
:10056000863038F085E0A2E0B0E0082E0E945B56AD
:1005700008958823C1F70895A2E0B0E00E94535681
:10058000902D892F8150853018F4892F90E008959F
:1005900083E00E94B00283E090E008958091D70745
:1005A000E82FF0E0EE0FFF1FEB55F84F80819181AF
:1005B0008D5E9F4F14F010920201808191818A5BC1
:1005C0009F4FACF480910201882389F481E08093ED
:1005D000020120919A062F5F20939A06253050F051
:1005E00088EE93E09093E6038093E50308C02091A2
:1005F0009A0605C0822F0E94033520919A06822F09
:1006000090E090936807809367070895582F9B01A7
:10061000863060F5882349F1A82FB0E01197842F28
:1006200090E0BD01689FD001699FB00D789FB00D2B
:100630001124AC59BF4FF901019724F001900E9499
:100640005B56FACF62E670E0DB01042E0E945B5637
:1006500088E062517040DB01F901182E0E94675654
:10066000852F0E94B0020E94C351089555E0A4E076
:10067000B0E0D5CFA82FFB018150853018F0A2E063
:10068000B0E002C0B0E01197842F90E09D01289F58
:10069000D001299FB00D389FB00D1124AC59BF4F28
:1006A000019724F00E9453560192FACF0E94C35141
:1006B00008952F923F924F925F926F927F928F9206
:1006C0009F92AF92BF92CF92DF92EF92FF920F93E1
:1006D0001F93CF93DF93CDB7DEB722970FB6F89471
:1006E000DEBF0FBECDBF14B815B8189BF8C2199B5A
:1006F000F2C28DE08093000181E887B93E9A8FEFC6
:1007000088B98BE184B981E085B98EE38AB9579ABB
:1007100087E48BB9469A84B7877F84BF8091600055
:100720008861809360001092600080ED97E0909364
:10073000E6038093E50310929A04109299041092B4
:10074000AA071092A9071092980410929704109289
:1007500096041092950420910001243108F4C5C23A
:1007600088E894E0A0E0B0E08093B3039093B403F2
:10077000A093B503B093B6032A3009F48BC2243199
:1007800009F488C2289A0E94E6120E94BE120E94B2
:1007900065080E94C2220E94F9150E94AD210E94A4
:1007A0008D4E789420910001822F6AE00E94E355DB
:1007B000492F50E0822F0E94E35590E020E730E07F
:1007C0003F932F9328E430E03F932F931F921F9283
:1007D0005F934F939F938F9382EB91E09F938F93BF
:1007E0001F920E94C30E8091C8002DB73EB7235FB1
:1007F0003F4F0FB6F8943EBF0FBE2DBF803209F4B5
:1008000020C281E991E09F938F931F920E94C30EB3
:100810000F900F900F90809100018C3008F00FC264
:10082000299A49E067ED77E083E00E943A0371E09E
:10083000C72E70E0D72ED6010E945356802D8A34E1
:1008400009F4B2C00E947F3682E891E09F938F93B3
:100850001F920E94C30E1A8219820F900F900F9060
:1008600060E5A62E60E0B62E51E5852E50E0952E6F
:1008700042E5642E40E0742E33E5432E30E0532EE3
:1008800024E5222E20E0322E97E5E92E90E0F92E85
:100890000981102F1F5F123009F4C1C1133009F410
:1008A000FBC1143008F0BBC180910001843168F0B5
:1008B00085E08093EF07109207088BE18093EB07A8
:1008C0008EE48093040880930508D5010E94535656
:1008D000802D8C3008F05DC0D4010E945356802DCD
:1008E0008C3008F056C0D3010E945356802D8C30B6
:1008F00008F04FC0D2010E945356802D8C3008F072
:1009000048C0A0E5B0E00E945356802D8093D707E1
:10091000A1E5B0E00E945356802D8093D807A2E550
:10092000B0E00E945356802D8093D907A3E5B0E034
:100930000E945356802D8093DA07D1010E945356AE
:10094000802D8093DB07A5E5B0E00E945356802DF3
:100950008093DC07A6E5B0E00E945356802D80937B
:10096000DD07D7010E945356802D8093DE0711309A
:1009700009F495C14CE567ED77E0812F0E940603ED
:100980000E5F063048F489819A8101969A838983A3
:100990007FCF0E94C423EECF83E00E94B0028AE49E
:1009A000D601082E0E945B56A4E0B0E00E94535688
:1009B000802D853008F084C10E94BC024CE567EDB3
:1009C00077E00E943A030E94BC0290E09F938F93CD
:1009D00086E191E09F938F931F920E94C30E8091B6
:1009E000DF070F900F900F900F900F9080FD31C197
:1009F00008EE13E00E948632809100018A3009F4EB
:100A00001CC1843109F419C1289A80ED97E09093B4
:100A1000E6038093E50385E580939C0686EE90E0EF
:100A20009F938F931F920E94C30E8091DF070F90B8
:100A30000F900F9082FFF6C08AED90E09F938F9306
:100A40001F920E94C30E0F900F900F908EEC90E0BB
:100A50009F938F931F920E94C30E0E94581B88E899
:100A600093E1909394038093930381E080939B069A
:100A70000F900F900F908091E203882309F471C0CA
:100A800080911D03882309F46CC01092E2038091C9
:100A90009A06882309F471C00E94CE020E94C430D5
:100AA000209100012A3009F471C0243109F46EC08C
:100AB000289A80910501882309F46EC081508093A3
:100AC000050180919404882329F080919404815039
:100AD000809394048091930390919403892B09F45B
:100AE0006CC0809193039091940301979093940329
:100AF000809393032A3009F45EC0243109F45BC06B
:100B0000289A8091E203882329F080919D0488230C
:100B100009F075C00E94A4090E94350CC8010E940A
:100B20008E128823E1F020910E0330910F03809103
:100B3000F00790E02817390744F480910903909159
:100B40000A038F5F9F4F09F45DC00E94F85084E054
:100B50008093E70384E190E00E9485128C010E945B
:100B6000D2518091E703882309F085CF0E94395143
:100B70008091E2038823A9F383CF0E942E370E943D
:100B8000C430209100012A3009F08FCF289880913D
:100B90000501882309F092CF1092A6061092B504A1
:100BA0001092B4041092B7041092B6041092B904D3
:100BB0001092B80486CF2898A4CF85E090E0909357
:100BC0009403809393030E94C7218091090390911D
:100BD0000A038F5F9F4F09F094CF80919D04882373
:100BE00009F48FCF80E197E29093E6038093E503C9
:100BF00080E890E090930A038093090382CF0E94DB
:100C0000350C8CCF80E797E19093E6038093E50362
:100C100080E093E090930A038093090396CF0E94AB
:100C2000CE3542CE82ED90E09F938F931F920E942B
:100C3000C30E0F900F900F9009CF2898E6CE2998F9
:100C4000F0CD8091CA00863009F0DBCD0E948C5235
:100C5000D8CD89EF90E09F938F931F920E94C30E8F
:100C600088EE93E00E9485128C010E94FC1A0F907E
:100C70000F900F90C8010E948E128823D9F384EF41
:100C800090E09F938F931F920E94C30E0F900F903E
:100C90000F90B0CE289877CD0E941F3505CEEAE49C
:100CA000F1E0FF93EF931F920E94C30E4CE567EDB6
:100CB00077E081E00E9406030F900F900F9063CEC3
:100CC00081E391E09F938F931F920E94C30E0F9038
:100CD0000F900F9071CE8BE0809300010DCD199B8A
:100CE00011C084E18093000107CD8BE095E0A0E086
:100CF000B0E08093B3039093B403A093B503B09393
:100D0000B6033ACD8AE080930001F6CC1F920F9291
:100D10000FB60F9211248F939F93EF93FF938091BF
:100D200003018823A9F48091DE039091DF030196EB
:100D30009093DF038093DE03FC01E45AFA4FE081D5
:100D4000ED3059F08639910541F0E093C6000DC0B1
:100D50001092DF031092DE0308C01092DF0310929E
:100D6000DE0381E080930301F0CFFF91EF919F912B
:100D70008F910F900FBE0F901F9018951F920F929A
:100D80000FB60F9211242F933F934F938F939F93FE
:100D9000AF93BF93CF93DF93EF93FF938091C60000
:100DA0008093C9034091D903463910F01092D803BB
:100DB0008091C9038D3009F18091D803813009F405
:100DC00090C0813030F0823009F473C01092D803A3
:100DD000B5C08091C903833209F4A1C08091C903D1
:100DE0008093A90681E08093D9038091C90390E0A4
:100DF0009093DD038093DC03A1C08091D8038230FF
:100E0000E9F61092D803A42FB0E0FD01E955F94F9F
:100E10003081ED01C855D94F28818091DC03909134
:100E2000DD03831B9109821B91099F709093DD0361
:100E30008093DC039C010024220F331F001C220F2F
:100E4000331F001C232F302D235C2093DB03982FAE
:100E50009F73935C9093DA038081281709F468C02C
:100E60008091CC038F5F8093CC0390E08091CA0384
:100E7000882309F063C0992309F460C081E080935E
:100E8000CA034F5F4093CD03A755B94F8DE08C93B4
:100E90008091AB06823509F051C088E190E02CE0EA
:100EA0000FB6F894A895809360000FBE2093600061
:100EB00045C0E42FF0E08091C903E755F94F8083E6
:100EC000463948F11092D8032091C9038091DC0380
:100ED0009091DD03820F911D9093DD038093DC03DD
:100EE0002DC082E08093D803E42FF0E08091C90305
:100EF000E755F94F80834F5F4093D9032091C90391
:100F00008091DC039091DD03820F911D9093DD03AE
:100F10008093DC0313C04F5F4093D903D5CF8091FA
:100F2000CA03882309F05ACF81E08093D80356CFB3
:100F30008881981709F094CF91E098CFFF91EF91B5
:100F4000DF91CF91BF91AF919F918F914F913F9141
:100F50002F910F900FBE0F901F901895CF93DF9396
:100F6000BC01892B19F120E030E040E050E0FA01AB
:100F7000E45AFA4F8081280F311D4F5F5F4F4617AB
:100F80005707A9F73F70C9010024880F991F001C5B
:100F9000880F991F001C892F902D835CDB0111960F
:100FA0002F73235CED012196FB0108C0E0E0F0E027
:100FB0008DE3A1E0B0E02DE3C2E0D0E0E45AFA4FC7
:100FC0008083A45ABA4F2C93C45ADA4F8DE0888399
:100FD0001092030180915C058093C600DF91CF9150
:100FE00008954091CD03465009F451C033E063E0C9
:100FF00030C0282F2D53E62FF0E0822F82958F707E
:101000009D53990F990F982BE755F94F9083E62F31
:10101000EF5F4130D1F1972F9D53F0E02295207F73
:10102000892F86958695282BE755F94F2083E62F43
:10103000EE5F43504F3F49F1F0E09295990F990FC1
:10104000907C5D53952BE755F94F90836D5F44235A
:10105000D9F0E32FF0E0E755F94F90813F5FE32FA0
:10106000F0E0E755F94F80813F5FE32FF0E0E7556F
:10107000F94F70813F5FE32FF0E0E755F94F508162
:101080003F5F442309F0B5CFE62FE35001C0E0E015
:101090008CEA96E09093CF038093CE03E093D00345
:1010A00008951F93182F8A3029F08091C00085FF82
:1010B000FCCF04C08DE00E945108F7CF1093C6000A
:1010C00080E090E01F9108950895E1ECF0E088E160
:1010D0008083A0ECB0E08C9182608C9380818068EA
:1010E00080838081806480838AE28093C4008091C1
:1010F0000701909108010E948512909389068093C0
:1011000088068CED90E00E9485129093A80680934B
:10111000A70610928A0688E480938B068FE080935E
:101120008E068AE080938C0610928D061092CF0373
:101130001092CE031092D0030895EF92FF920F9376
:101140001F93CF93DF93CDB7DEB722970FB6F894F6
:10115000DEBF0FBECDBF9C854D8583E280935C05CD
:101160009F5990935D058B8580935E05CE010E9609
:101170009A838983442319F463E070E0D5C00E8517
:101180001F85CE0142969A83898328893989211542
:10119000310591F3F42EFA9463E070E0A0E05EC0B4
:1011A000EA2FF0E0AF5FC901E00FF11F40819C0121
:1011B0002150304009F473C0EA2FF0E0AF5FE00F38
:1011C000F11FB0812150304009F079C0FF2009F4AF
:1011D00076C0E981FA81008111813496FA83E9832E
:1011E000349722813381FA94842F90E042954F7096
:1011F0008F7090705B2F5295569556955370880F4F
:10120000991F880F991F582B535CBF73B35CA0E0E4
:101210008E2D86958695835CFB01E45AFA4F808378
:101220008E2D90E08370907082959295907F982794
:10123000807F9827482B435CFB01E35AFA4F408399
:10124000FB01E25AFA4F5083FB01E15AFA4FB08397
:101250006C5F7F4F2115310509F466C0F801EA0F74
:10126000F11DE080AF5F2150304009F099CFFF20A1
:1012700091F0E981FA81008111813496FA83E98342
:10128000349782819381FA94009721F0E0E0F0E0B6
:10129000A1E08ACFA0E040E05DE3BDE3B9CFFF204D
:1012A00011F5842F90E042954F708F709070880FE9
:1012B000991F880F991F582F535CBDE3A9CF842F26
:1012C00090E042954F708F7090705B2F52955695BD
:1012D00056955370880F991F880F991F582B535C90
:1012E000BF73B35C95CFE981FA8100811181349697
:1012F000FA83E983349722813381FA9421153105E9
:1013000079F4842F90E042954F708F709070880F21
:10131000991F880F991F582F535CA0E0BDE378CF29
:10132000E0E0F0E0A1E04BCFCB010E94AE072296B7
:101330000FB6F894DEBF0FBECDBFDF91CF911F91E6
:101340000F91FF90EF900895EF92FF920F931F93EC
:1013500080910301882309F483C28091C403882308
:1013600029F080910301882309F04AC18091C303C9
:10137000882329F080910301882309F07BC18091A3
:10138000C603882329F080910301882309F0A2C1B4
:101390008091C203882329F080910301882309F0FA
:1013A000B9C18091A7069091A8060E948E12882349
:1013B00029F080910301882309F0D1C180910701B0
:1013C00090910801892B09F06DC08091C503882395
:1013D00029F080910301882309F0EAC08091D603A7
:1013E0009091D703892B09F06CC0809104018F3F45
:1013F00059F190E082959295907F9827807F982769
:10140000875F9E4F20E130E03F932F939F938F9310
:1014100081E090E09F938F9384E091E09F938F937E
:1014200082E08F9381E08F9381E48F930E949D08E7
:101430008FEF809304012DB73EB7255F3F4F0FB666
:10144000F8943EBF0FBE2DBF80918107882329F0FD
:1014500080910301882309F0E5C18091C7038823A7
:1014600009F4FEC180910301882309F4F9C186E1E2
:1014700090E09F938F9385EA97E09F938F9381E00D
:101480008F938F9380E58F930E949D081092C703DE
:101490002DB73EB7295F3F4F0FB6F8943EBF0FBE42
:1014A0002DBFDEC180918806909189060E948E1220
:1014B000882309F48ACF80910301882309F48ECF11
:1014C00077C080915A0590915B050E948E12882307
:1014D00009F48BCF80910301882309F486CFE09033
:1014E000EB07FF24EE0CFF1CEE0CFF1C0027F7FCA3
:1014F0000095102F60914504709146048091470437
:1015000090914804A80197010E94385630934D05E8
:1015100020934C0560914D0470914E0480914F04CE
:1015200090915004A80197010E94385630934F05BE
:1015300020934E0560917E0870917F08809180080D
:10154000909181082AE030E040E050E00E94C455CC
:101550002091B3033091B4034091B5035091B60389
:101560000E94385630935105209350058EE090E04C
:101570009F938F938CE495E09F938F9381E08F935B
:101580008F9383E48F930E949D088091D60390915E
:10159000D7030E94851290935B0580935A058DB7FF
:1015A0009EB707960FB6F8949EBF0FBE8DBF1DCF96
:1015B00082E490E09F938F938FE397E09F938F93C4
:1015C00081E08F938F9384E48F930E949D08109203
:1015D000C50380910701909108012DB73EB7295F9F
:1015E0003F4F0FB6F8943EBF0FBE2DBF009709F4D2
:1015F000F5CE0E9485129093890680938806EECEE0
:101600000E94611B8091C80324E1829FC0011124C4
:10161000885D9C4F24E130E03F932F939F938F93FD
:1016200081E090E09F938F9388EC93E09F938F935A
:1016300082E08F9381E08F9388E48F930E949D08CE
:101640008091C8038F5F8093C8032DB73EB7255F95
:101650003F4F0FB6F8943EBF0FBE2DBF843010F041
:101660001092C8031092C4038091C303882309F425
:1016700086CE80CE0E94611B80E590E09F938F9381
:1016800088E293E09F938F9321E030E03F932F9384
:1016900088E793E09F938F933F932F9386E294E0A4
:1016A0009F938F9383E08F9381E08F938CE48F934C
:1016B0000E949D081092C3038DB79EB70F960FB678
:1016C000F8949EBF0FBE8DBF8091C603882309F496
:1016D0005FCE59CE8AE090E09F938F938AE896E0A0
:1016E0009F938F9381E08F938F9386E58F930E94D2
:1016F0009D081092C6032DB73EB7295F3F4F0FB626
:10170000F8943EBF0FBE2DBF8091C203882309F419
:1017100048CE42CE209106018BE090E09F938F93BC
:101720008CE996E09F938F9381E08F932F9387E4CA
:101730008F930E949D081092C2038DB79EB70796A3
:101740000FB6F8949EBF0FBE8DBF8091A7069091F3
:10175000A8060E948E12882309F430CE2ACEE0908B
:10176000EB07FF24EE0CFF1CEE0CFF1C0027F7FC20
:101770000095102F609145047091460480914704B4
:1017800090914804A80197010E943856309395061D
:101790002093940660914D0470914E0480914F0403
:1017A00090915004A80197010E94385630939706F3
:1017B000209396068091AC04809398068091AD04A6
:1017C0008093990688E090E09F938F9384E996E058
:1017D0009F938F9381E08F9383E08F9387E78F931D
:1017E0000E949D082DB73EB7295F3F4F0FB6F89472
:1017F0003EBF0FBE2DBF80919A06853018F086E05F
:1018000080939A0683E690E00E9485129093A80642
:101810008093A7068091070190910801892B09F414
:10182000D4CD40CE81E090E09F938F9381E897E004
:101830009F938F9381E08F938F9382E48F930E9485
:101840009D08109281078DB79EB707960FB6F89442
:101850009EBF0FBE8DBF8091C703882309F002CEC3
:101860001F910F91FF90EF900895EF92FF920F93C9
:101870001F93CF93DF93CDB7DEB722970FB6F894BF
:10188000DEBF0FBECDBF8091CA03882309F415C205
:101890000E94F1078091AA06823679F18091AB0609
:1018A000843609F449C18536C0F18C3609F429C162
:1018B0008D3608F072C0873609F4E9C08836A1F485
:1018C0008FEF8093050180912704E091CE03F09182
:1018D000CF039081892B80932704882311F01092E5
:1018E000C80381E08093C4031092CA031092CF030F
:1018F0001092CE031092D003E0C18091AB068137E5
:1019000009F476C0823770F58B3409F429C1803729
:1019100029F681E08093C703C1CF813609F4FFC067
:10192000823608F044C08B34F9F6E091CE03F09192
:10193000CF03808191819093820480938104845E9F
:101940009D4F2091830430918404821B930B68E6A1
:1019500071E00E940356845B9040909386048093CC
:101960008504C2CF833709F419C1843709F096CFB3
:101970000091CE031091CF03F80180819181A28163
:10198000B3818093D2039093D303A093D403B093F5
:10199000D5038FEF8093050181CF843709F48EC082
:1019A000863709F0A1CF81E08093C6039DCF8236B0
:1019B00009F471C0833609F097CF8091D6039091D6
:1019C000D703892B09F051C10091CE031091CF03A9
:1019D000F8019081992309F058C1F80180812AE02B
:1019E000829FC00111249093D7038093D6037CCFAC
:1019F0000091CE031091CF03F80180818F3F09F44D
:101A000053C1F8018081882309F034C181E08083CB
:101A10000091CE031091CF0397EDE92E97E0F92EB8
:101A20004CE5B701F80180810E943A0380910301DF
:101A30008823E1F3E091CE03F091CF038081898385
:101A40008AE48A838CE590E09F938F93FF92EF92D4
:101A500021E030E03F932F93CE0102969F938F9326
:101A60003F932F93CE0101969F938F9383E08F93A3
:101A700081E08F9381E58F930E949D088DB79EB77B
:101A80000F960FB6F8949EBF0FBE8DBF07CF81E0B3
:101A90008093C20329CFACE9B6E0E091CE03F09188
:101AA000CF038BE001900D928150E1F78091A50664
:101AB000809381078FEF8093050116CFE091CE03CD
:101AC000F091CF0380819181A281B3818093D20371
:101AD0009093D303A093D403B093D50380910301D3
:101AE0008823E1F3809106011F928F9384E58F9301
:101AF0000E949D088FEF809305010F900F900F902B
:101B0000F3CE8FEF80930501E091CE03F091CF03E8
:101B100080818093260481E08093C303E5CEE09129
:101B2000CE03F091CF03808180930401803210F2C4
:101B30008FE180930401BECFE091CE03F091CF03FB
:101B400080812AE0829FC001112490930801809334
:101B50000701892B09F4C8CE81E08093C503C4CE68
:101B60000091CE031091CF03F80180819181909371
:101B7000820480938104845E9D4F20918304309180
:101B80008404821B930B68E671E00E940356845B19
:101B90009040909386048093850480CE0091CE037C
:101BA0001091CF03F80180818150853018F4818134
:101BB0008A34E9F01982809103018823E1F381E0FE
:101BC00090E09F938F93CE0101969F938F9381E036
:101BD0008F938F9383E58F930E949D088DB79EB757
:101BE00007960FB6F8949EBF0FBE8DBF57CEA7EDD8
:101BF000B7E032968CE501900D928150E1F74CE50B
:101C000067ED77E0F80180810E9406036091040887
:101C100070E080E090E024EC39E040E050E00E9489
:101C2000C45560939703709398038093990390939E
:101C30009A036091050870E080E090E00E94C4552E
:101C400060939B0370939C0380939D0390939E03EA
:101C5000E091CE03F091CF0380810E94B0020E94F8
:101C6000BC0289830E940335A6CF0091CE03109158
:101C7000CF03B3CE863008F4CFCE85E0F801808361
:101C80000091CE031091CF03C7CE8AE0989FC00188
:101C900011240E94851290935B0580935A05009150
:101CA000CE031091CF0399CE0E94BC02F80180832D
:101CB0000091CE031091CF03A4CE22960FB6F894D4
:101CC000DEBF0FBECDBFDF91CF911F910F91FF906F
:101CD000EF900895982F80918207813031F0892FFD
:101CE0000E945108282F30E00CC080912504E82F75
:101CF000F0E0E85DFC4F90838F5F8093250421E046
:101D000030E0C90108951F93182F18162CF480E3B2
:101D10000E946A0E1150D9F71F9108951F93182F32
:101D200018162CF480E20E946A0E1150D9F71F9108
:101D300008950F931F93CF93DF938C01EB01672BD3
:101D400049F0F8010F5F1F4FE4918E2F0E946A0E39
:101D50002197B9F7DF91CF911F910F9108950F93BC
:101D60001F93CF93DF938C01EB01672B39F0F801C0
:101D700081918F010E946A0E2197C9F7DF91CF915F
:101D80001F910F9108952F923F924F925F926F9201
:101D90007F928F929F92AF92BF92CF92DF92EF92FB
:101DA000FF920F931F93CF93DF93CDB7DEB7E597E5
:101DB0000FB6F894DEBF0FBECDBF2B968FAD2B971D
:101DC00080938207CE01835B9F4F9B838A832D96EE
:101DD0000EAD1FAD2D971EA61FA618AA19AAF801B1
:101DE0008491882309F4A2C2853209F41BC26801D8
:101DF00003C0F5E2FF1639F00894C11CD11CF601AE
:101E0000F490FF20B1F7B601601B710B19F0C80107
:101E10000E94990EFF2009F489C286010F5F1F4FAF
:101E20001982AA81BB818EA49FA4A8A8B9A8332433
:101E300022248FEF8BABF8010F5F1F4FF490C32C60
:101E4000DD2491E0C922DD24E5E7FE1609F443C054
:101E50008F2D8062883709F43EC0F0E2FF1609F446
:101E600048C083E2F81609F48FC0EAE2FE1609F4CE
:101E700080C0FDE2FF1609F482C0EBE2FE1609F411
:101E80003CC0FEE2FF16D9F180E3F81609F47FC0EA
:101E90008F2D8153893008F07FC020E030E0C901E8
:101EA000880F991F880F991F880F991F220F331FC2
:101EB000280F391F2F0D311D20533040F8010F5FBF
:101EC0001F4FF4908F2D80538A3048F3222EE5E780
:101ED000FE1609F0BDCFC114D10409F43CC08D90A9
:101EE0009D90AD90BC9013971496F0E2FF1609F008
:101EF000B8CF8981882309F09ECFF9829CCFF80161
:101F00000F5F1F4F94919A3209F44FC0892F80536D
:101F10008A3060F5492F20E030E0C901880F991F11
:101F2000880F991F880F991F220F331F280F391F01
:101F3000240F311D20533040F8010F5F1F4F649173
:101F4000462F862F80538A3040F3A90137FD0BC0FE
:101F50004BABF62E79CF8D919C9111974C01AA2411
:101F6000BB2412967ACF4FEF5FEFF2CFF92E1BAA68
:101F70006BCFFD011296208027FE5DCF219480E17A
:101F8000382A9FED392257CF98E0392A54CF34FCB4
:101F900052CF90E2392A4FCFE8E6FE1679F08CE670
:101FA000F81679F491E0392A46CFCD0102964D9189
:101FB0005C9157FD77C04BABDC013DCFF4E03F2A8D
:101FC0003ACFBB83AA83E3E6FE1609F40BC1F4E41F
:101FD000FF1609F46AC084E6F81609F468C099E6A9
:101FE000F91609F464C09FE4F91609F407C1EFE695
:101FF000FE1609F4FFC0E0E7FE1609F45DC193E7A1
:10200000F91609F419C185E5F81609F410C195E728
:10201000F91609F409C198E5F91609F469C1E8E768
:10202000FE1609F465C1FF2009F480C1FE82198201
:10203000632C77248EA69FA6A8AAB9AAEE2436E020
:10204000C32ED12CCC0EDD1E81E0E1E090E021E03A
:10205000A22EB12C2981222309F4A0C08F5F582E13
:10206000590E40E3842E912C8620972081149104F0
:1020700009F438C1222309F02EC166FCC9C0F0E280
:102080008F16910409F4BFC08E2D0E94830EB501F6
:10209000C6010E94AF0E64FEA2CE822D85190E9459
:1020A0008E0E9DCE4FEF5FEF86CFE1E03E2A30FEF1
:1020B0008EC01496BB83AA83BE90AE909E908E90E5
:1020C000B7FC78C0FAE0FAABEBA9E7FD02C0FFED80
:1020D0003F2281149104A104B104A9F18AA9482ED8
:1020E000552466247724EEE2CE2ED12CCC0EDD1EB4
:1020F000DDAACCAA17C070E3E72EE60EF601E29245
:102100006F01C501B401A30192010E9416562EA7CA
:102110003FA748AB59AB84149504A604B704A0F1BB
:1021200049015A01C501B401A30192010E9416564A
:102130006A3008F357E5E52EE60EF8E5FF16F1F6EE
:102140008FEDE822DBCF9BA99923C1F4632C772480
:102150001EA61FA618AA19AAFEE2CF2ED12CCC0EBD
:10216000DD1E80E0E0E04BA9E42EEE1AE7FC1BC088
:102170009E2DA82EBB24A7FCB0946CCFEAA94E2EAE
:10218000552466247724AFCFFAA9F83009F4BCC0EF
:10219000ECA9EC198E2F632C7724E5CF66FE5FCF78
:1021A0008E2F8E5F5CCFA82EBB24A7FCB094EE24AC
:1021B00090E050CFB094A09490948094811C911C96
:1021C000A11CB11C2DE229838AE08AAB7DCF129637
:1021D000BB83AA839E918E914C01AA2497FCA09464
:1021E000BA2C6ECF1296BB83AA8312978C918E83E2
:1021F00019821ECFF8E0FAAB198266CF81E0382A47
:1022000098E09AABF9CF822D85190E94830E3CCFBE
:1022100080E38C83FD8262E070E0CE0104960E9430
:10222000AF0E2DCF6801F9CDEAE0EAABE5CFF1E0E2
:102230003F2A8AE08AABE0CF1296BB83AA83DE9066
:10224000CE90C114D10489F488E28E838EE68F8308
:1022500085E788878CE689878A8789E28B871C8651
:10226000A6E0CA2ED12CCC0EDD1EEBA9E7FD1CC0CA
:102270004E2F552747FD509560E070E0C6010E9443
:102280006754009779F08C19FBA9F8170CF48F2F7D
:102290001982E82F632C77248EA69FA6A8AAB9AA34
:1022A00040E062CF8BA9F4CFF60101900020E9F75E
:1022B00031978E2F8C19ECCF1296BB83AA839E91F7
:1022C0008E914C01AA24BB24F0E43F2AB8E7FB2EF0
:1022D00080E18AAB91CF61E070E0CE0101960E946F
:1022E000AF0ECDCE822D85190E948E0E2981C2CED1
:1022F00033FE19C081149104A104B104A1F0F0E4EB
:102300003F2A80E18AAB78CF632C772433FE07C065
:1023100080E3E81621F080E3F60182936F01ECA9D7
:10232000EC198E2F20CF90E19AAB66CFE5960FB6D1
:10233000F894DEBF0FBECDBFDF91CF911F910F91FB
:10234000FF90EF90DF90CF90BF90AF909F908F90D5
:102350007F906F905F904F903F902F9008951F92C5
:102360000F920FB60F9211242F933F935F936F93A9
:102370007F938F939F93AF93BF938091E7038823BD
:1023800029F08091E70381508093E7038091F50362
:1023900081508093F5038F3F09F488C08091E50355
:1023A0009091E6030297E0F08091E5039091E603B7
:1023B00001979093E6038093E5038091E503909164
:1023C000E6032091090330910A0382239323892B8A
:1023D00069F0809100018A3009F482C0479A0CC0EC
:1023E0008FEF9FEF90930A03809309038091000180
:1023F0008A3009F473C047988091DF0783FF77C064
:10240000349B0AC08091E3039091E403019690937A
:10241000E4038093E3036BC08091E3039091E403B2
:10242000892B49F18091E3039091E4038A5691400E
:1024300010F58091E3039091E4032091E303309140
:10244000E40369E270E00E94EF55260F371F3093D6
:10245000E4032093E3038091E3039091E4030B975B
:1024600008F440C08091E3039091E4030A979093AD
:102470008204809381048091810490918204845E1F
:102480009D4F2091830430918404821B930B68E656
:1024900071E00E940356845B904090938604809381
:1024A00085041092E4031092E30321C089E0809335
:1024B000F50380910D038F5F817080930D03882356
:1024C00019F481E08093E2038091E0039091E103AD
:1024D00001969093E1038093E00360CF5A988CCFEC
:1024E0005A9A8ACF1092820410928104C4CFBF916D
:1024F000AF919F918F917F916F915F913F912F91BC
:102500000F900FBE0F901F9018952091E00330910F
:10251000E1032F5F3F4F820F931F08952091E00347
:102520003091E103821B930B892F99278695807444
:1025300090E00895CF93DF930E948512EC01CE01C5
:102540000E948E128823D9F3DF91CF910895CF9303
:10255000DF930E948512EC0109C080911D0388233E
:1025600029F010921D038FEC80937A00CE010E9417
:102570008E12882391F3DF91CF9108959FB7F8943D
:10258000579A5F983E9A469AA0EBB0E08C918F7074
:102590008C938C9183608C93E1EBF0E080818B7362
:1025A000808380818B6080831092B2008FEF809354
:1025B000B3008C9180688C93E0E7F0E080818A7FA3
:1025C00080838081826080839FBF08958AE090E04D
:1025D0000E9485129093F7038093F60382E085BDF5
:1025E00083EA84BD17BC88E788BD86E086BDEEE639
:1025F000F0E080818160808308951F920F920FB672
:102600000F921124CF92DF92EF92FF920F931F93BC
:102610002F933F934F935F936F937F938F939F93EA
:10262000AF93BF93EF93FF93809100018431B8F48F
:102630008091F403882309F45DC02091F203309166
:10264000F30341E02F373407C8F18FEF8093B300D5
:102650002F5F30403093F3032093F203B3C2809195
:10266000F403882351F78091B00086FF15C1809153
:10267000B0008F7B8093B000E091EF03EE2309F070
:1026800049C18091FD0790E02DED36E0A901849FBE
:102690009001859F300D949F300D11248091F0039F
:1026A0009091F103281B390B3093F3032093F2032D
:1026B0001092F1031092F003469AEAC02F3F3105C1
:1026C00081F078F051E02E37350709F414C180E825
:1026D0008093B300205830403093F3032093F203EB
:1026E00071C22093B3001092F3031092F203109280
:1026F000F40368C28091B00086FFAEC08091B00044
:102700008F7B8093B0008091AB03482F50E0440F43
:10271000551F440F551F20910B0330910C03C90125
:10272000880F991F820F931F480F591F57FD10C222
:10273000CA01959587959595879590930C038093FD
:102740000B039093EC038093EB038091230880FFAD
:1027500024C1C090EB03D090EC03E090FA07FF2473
:1027600000E010E0609145047091460480914704B8
:102770009091480420E830E040E050E00E94385654
:10278000C801B7010E94C455660F771F881F991FA3
:10279000660F771F881F991F20E031E040E050E06E
:1027A0000E943856C20ED31ED092EC03C092EB03A7
:1027B0008091FB07282F30E0220F331F220F331F99
:1027C0008091EB039091EC03821793070CF49DC06A
:1027D0008091FC07282F30E0220F331F220F331F78
:1027E0008091EB039091EC03281739070CF48DC00E
:1027F0002091EB033091EC0327553E4F3093F303C8
:102800002093F2038091EB039091EC0397FDA3C119
:1028100095958795959587959093EC038093EB0319
:102820008091EB039091EC0390936A078093690782
:1028300045E02D3D340708F4A5C02CED35E030937C
:10284000F3032093F2032091F2033091F3033093CA
:10285000F1032093F0031CC08091B000806480934A
:10286000B0008091FD0790E02DED36E0A901849F36
:102870009001859F300D949F300D11248091F003BD
:102880009091F103281B390B3093F3032093F2034B
:1028900081E08093F403D5CE8091B0008064809372
:1028A000B0002CEB30E03093F3032093F2038091DF
:1028B000F0039091F10384549F4F9093F103809320
:1028C000F0038091E803882329F080919404853BEC
:1028D00008F098C08091EF038F5F8093EF03909191
:1028E000FD07981708F089C01092EF032091F203BA
:1028F0003091F303CDCF8FEF8093B3002FE730E01B
:102900003093F3032093F2035DC13093EC032093E3
:10291000EB036ECF29EA33E03093F3032093F20305
:10292000E13009F471C0F0E0EE0FFF1FEB55F84FF6
:1029300080819181880F991F87559C4F9093F30355
:102940008093F2032091F2033091F30355E02D3D83
:10295000350708F4F1C02CED35E03093F3032093F4
:10296000F2032C5B30403093F3032093F203809109
:10297000F0039091F103820F931F9093F1038093E2
:10298000F00386CF2757314008F05DCF27E731E0CD
:102990003093F3032093F20356CFC090EB03D09013
:1029A000EC03E090FA07FF2400E010E0609145049A
:1029B00070914604809147049091480420E830E0EB
:1029C00040E050E00E943856C801B7010E94C4554B
:1029D000660F771F881F991F660F771F881F991F23
:1029E00020E031E040E050E00E943856C21AD30A9D
:1029F000D092EC03C092EB03DBCE2091F203309136
:102A0000F30346CF469866CF8091AB03482F50E042
:102A1000440F551F440F551F20910B0330910C0399
:102A2000C901880F991F820F931F480F591F57FD27
:102A3000C6C0CA01959587959595879590930C0387
:102A400080930B039093EC038093EB038091230816
:102A500080FF83C0C090EB03D090EC03E090FA07B6
:102A6000FF2400E010E060914504709146048091DD
:102A700047049091480420E830E040E050E00E9494
:102A80003856C801B7010E94C455660F771F881FCA
:102A9000991F660F771F881F991F20E031E040E0E3
:102AA00050E00E943856C20ED31ED092EC03C09262
:102AB000EB038091FB07282F30E0220F331F220FFA
:102AC000331F8091EB039091EC03821793077CF006
:102AD0008091FC07282F30E0220F331F220F331F75
:102AE0008091EB039091EC032817390724F430937D
:102AF000EC032093EB038091EB039091EC0387555B
:102B00009E4F9093F3038093F2038091EB03909197
:102B1000EC0397FD52C09595879595958795909371
:102B2000EC038093EB038091EB039091EC03909383
:102B30006A078093690706CF81E02737380708F0D6
:102B400010CF27E731E03093F3032093F20309CF4E
:102B50004D5F5F4FEDCD03965BCEC090EB03D09001
:102B6000EC03E090FA07FF2400E010E060914504D8
:102B700070914604809147049091480420E830E029
:102B800040E050E00E943856C801B7010E94C45589
:102B9000660F771F881F991F660F771F881F991F61
:102BA00020E031E040E050E00E943856C21AD30ADB
:102BB000D092EC03C092EB037CCF0396ACCF4D5F79
:102BC0005F4F37CFFF91EF91BF91AF919F918F9161
:102BD0007F916F915F914F913F912F911F910F9135
:102BE000FF90EF90DF90CF900F900FBE0F901F904F
:102BF000189510927C008FEC80937A0008951F92B4
:102C00000F920FB60F921124DF92EF92FF920F9363
:102C10001F932F933F934F935F936F937F938F9364
:102C20009F93AF93BF93CF93DF93EF93FF93D09096
:102C300021048D2DD394D0922104E82FF0E0E231CD
:102C4000F10540F01092210482E0809322048093E9
:102C50007C00F3C3E25CFF4FEE0FFF1F0590F49181
:102C6000E02D0994809178009091790020911B04C7
:102C700030911C04280F391F30931C0420931B042F
:102C800081E0809322048091220480937C00DD20E7
:102C900009F4D3C38FEC80937A00CFC3DD24109264
:102CA000210481E080931D0380910E0490910F0414
:102CB000019690930F0480930E0420917800309138
:102CC00079008091930790919407820F931F9093BE
:102CD00094078093930780918B078F5F80938B0776
:102CE00080918B07853008F4B4C080919307909150
:102CF000940797FD7FC3959587959093940780934C
:102D000093078091780090917900909319038093B4
:102D1000180310928B0760910C0470910D04809140
:102D20000B04992787FD9095D82FCC27C81BD90B6A
:102D3000209187073091880780919307909194079D
:102D400040919E0450919F04281B390B241B350B86
:102D50002C0F3D1F8091A10390E0A901489F900195
:102D6000499F300D589F300D11248FE190E0AC0148
:102D7000649FC001659F900D749F900D1124280FD2
:102D8000391F37FDE6C23595279535952795359539
:102D90002795359527953595279530930D042093E4
:102DA0000C046091930770919407E0901403F090E5
:102DB00015030091160310911703882777FD80955E
:102DC000982FA8019701220F331F441F551F220F70
:102DD000331F441F551F220F331F441F551F2E1929
:102DE0003F09400B510B620F731F841F951F6C5FCF
:102DF0007F4F8F4F9F4F28E030E040E050E00E942F
:102E000038562093140330931503409316035093C0
:102E100017032091870730918807809114039091C0
:102E20001503A0911603B0911703C20FD31FC81B3F
:102E3000D90BD0939F04C0939E04809193079091E7
:102E4000940797FD84C295958795909394078093F6
:102E5000930782E08093220416CF609178007091EE
:102E60007900E0903F04F0904004009141041091FB
:102E70004204882777FD8095982F0E940C55A80161
:102E800097010E9474540E94D9547093090460936E
:102E90000804809108049091090402970CF45CC224
:102EA00060913F04709140048091410490914204EC
:102EB00020E030E84BE354E40E94475588239CF51A
:102EC00060913F04709140048091410490914204CC
:102ED0002AE037ED43EA5CE30E94755460933F04B7
:102EE0007093400480934104909342048091BE0407
:102EF0009091BF04845F9140B0F460913F04709161
:102F0000400480914104909142042DEC3CEC4CEC47
:102F10005DE30E94755460933F0470934004809376
:102F200041049093420481E080930A0480917800E8
:102F3000909179009093860780938507809108048B
:102F40009091090420917D0430917E0440917F048A
:102F500050918004AA2797FDA095BA2F820F931F46
:102F6000A41FB51F80937D0490937E04A0937F04DB
:102F7000B0938004E0907D04F0907E0400917F0483
:102F80001091800460917D0470917E0480917F0493
:102F90009091800420E034E040E050E00E943856F8
:102FA000E21AF30A040B150BE0927D04F0927E0402
:102FB00000937F041093800483E08093220463CE07
:102FC000809178009091790020911D0430911E0429
:102FD000280F391F30931E0420931D0484E0809332
:102FE000220451CE40910E0350910F03809178003E
:102FF000909179009A01220F331F240F351F63E04F
:1030000070E00E94EF55260F371F369527953695AD
:10301000279530930F0320930E0385E080932204BD
:1030200032CE809178009091790090932004809323
:103030001F0486E08093220426CE209178003091F0
:10304000790080913B0490913C04821B930B9093F8
:1030500084078093830780918307909184079093DE
:1030600016048093150487E0809322040CCE80918F
:103070007800909179002091390430913A04821BB4
:10308000930B90938F0780938E0780918E0790917A
:103090008F07909314048093130482E0809322049A
:1030A000F2CD209178003091790080911D049091AB
:1030B0001E04820F931F90931E0480931D04109290
:1030C0002204E1CD809100018A3009F420C18431CD
:1030D00009F4A0C1809178009091790020911F049B
:1030E00030912004820F931F909303048093020475
:1030F00086E080932204C7CD20917800309179003A
:1031000080913B0490913C04821B930B9093840725
:103110008093830780918307909184072091150401
:1031200030911604820F931F90930504809304043A
:1031300087E080932204A7CD809178009091790058
:103140002091390430913A04821B930B90938F079E
:1031500080938E0780918E0790918F0720911304A2
:1031600030911404820F931F9093070480930604F8
:1031700082E08093220487CD2091780030917900FD
:1031800080911B0490911C04280F391F30931C045C
:1031900020931B04809100018A3009F4D1C0220FD2
:1031A000331F220F331F30931C0420931B042091E4
:1031B0001B0430911C04C90137FD2AC195958795E0
:1031C00095958795959587959093FF038093FE033A
:1031D0008091190490911A04820F931F97FD16C1D4
:1031E0009595879590931A048093190420912F0444
:1031F00030913004821B930B909311038093100342
:103200008091F8039091F9032091100330911103FC
:10321000280F391F37FDF7C0359527953093F903EF
:103220002093F80381E0809322042DCD2091780033
:103230003091790080911D0490911E04280F391F50
:1032400030931E0420931D04809100018A3009F4FC
:1032500070C0220F331F220F331F30931E042093A0
:103260001D0420911D0430911E04C90137FDC9C001
:103270009595879595958795959587959093010454
:10328000809300048091170490911804820F931F7B
:1032900097FDB5C095958795909318048093170472
:1032A0002091310430913204821B930B90931303CD
:1032B000809312038091FA039091FB0320911203F3
:1032C00030911303280F391F37FD96C03595279588
:1032D0003093FB032093FA0383E080932204D3CC42
:1032E000809178009091790090931C0480931B0446
:1032F00081E080932204C7CC80917800909179007E
:1033000090931E0480931D0410922204BCCC8091E3
:10331000780090917900019620911F04309120044B
:10332000820F931F969587959093030480930204D0
:10333000DFCE220F331F30931E0420931D0491CF44
:10334000220F331F30931C0420931B0430CF0196AF
:103350007ACD215E3F4F17CD8091080490910904EA
:103360008F5F9F4F0CF0DFCD60913F047091400460
:10337000809141049091420420E030E849E054E417
:103380000E944B5518160CF0CECD60913F04709101
:10339000400480914104909142042AE037ED43EAD1
:1033A0005CE30E94745460933F04709340048093E4
:1033B0004104909342048091BE049091BF04845FC5
:1033C000914008F0B0CD60913F047091400480912D
:1033D0004104909142042DEC3CEC4CEC5DE30E94E6
:1033E000745460933F04709340048093410490931D
:1033F000420499CD01967FCC2F5F3F4F67CF019656
:1034000049CF079635CF2F5F3F4F06CF0196E8CEC5
:103410000796D4CE80917800909179002FEF37E015
:10342000281B390B80911F0490912004281B390B15
:1034300030930304209302045BCEFF91EF91DF9160
:10344000CF91BF91AF919F918F917F916F915F913C
:103450004F913F912F911F910F91FF90EF90DF902F
:103460000F900FBE0F901F9018950F931F931092FF
:10347000100410921104109212041CE800E00330B2
:1034800009F4A3C08091FE039091FF038C5F9340E9
:103490000CF08DC080911A03815080931A0300E0D4
:1034A00080910004909101048C5F93400CF072C0F5
:1034B00080911B03815080931B03809102049091A3
:1034C00003048C5F93400CF058C080911C03815022
:1034D00080931C0388E0809328040E94B32180918C
:1034E0001A038A3008F040C081E0809310048AE01B
:1034F00080931A0380911B038A3068F581E08093E2
:1035000011048AE080931B0380911C038A30D0F45D
:1035100081E0809312048AE080931C038091280448
:103520008823E1F710928B078FEC80937A008091CB
:103530008B078823E1F31A3008F442C0115009F0D8
:103540009ECF53C0863F50F381E08093120485EFF5
:1035500080931C03E3CF863FB8F281E0809311048F
:1035600085EF80931B03D0CF863F20F281E08093CC
:10357000100485EF80931A03BDCF809102049091CF
:1035800003048750944044F180911C038F5F809323
:103590001C03A0CF809100049091010487509440B7
:1035A000CCF080911B038F5F80931B0386CF8091AB
:1035B000FE039091FF038750944084F401E070CFA4
:1035C0008AE090E00E94A712B9CF1B3008F45ACFCE
:1035D00019E058CF0F5F71CF0F5F7CCF80911A0336
:1035E0008F5F80931A0300E05BCF86E490E00E9437
:1035F000A7121F910F910895CF92DF92EF92FF9241
:103600001F93CF93DF93F3E0EF2EF0E0FF2ED7016F
:103610000E945356802DC82FD0E0C531D10508F047
:103620002A97C7BD10920B0484E690E00E94A7126F
:1036300080911803909119038255934008F5C0E0DA
:10364000D0E0E6EECE2EE1E0DE2E04C02196CA3FA9
:10365000D105D8F41C2FC7BD82E390E00E94A712C9
:10366000DF92CF921F920E94C30E80911803909117
:1036700019030F900F900F908255934038F706C0B2
:1036800076EEC72E71E0D72EE5CF1C2FD701012E85
:103690000E945B56109390078CE291E00E94A71263
:1036A000DF91CF911F91FF90EF90DF90CF90089521
:1036B000E8E2F3E080E2819383E0E837F807D1F7AE
:1036C00008951F934091780380912604481710F4C1
:1036D0004093260480912704282F30E0C90181708F
:1036E0009070582F882341F080912604882309F494
:1036F000EAC0815080932604B9016270707021FF86
:1037000008C080912604481709F4E0C08F5F8093B9
:103710002604552319F0672B09F0D2C00E94581BCC
:10372000909126049A3068F581E180932504892FD1
:1037300090E09F938F938DE195E09F938F9381E02D
:103740008F930E94C30E0F900F900F900F900F90C9
:1037500010912604153009F4D7C31630E0F0183064
:1037600009F4EDC2193008F0B4C0163009F48BC268
:10377000173009F45EC2115010937803109226049A
:10378000E8C580E180932504892F90E09F938F9373
:1037900088E195E0D2CF123009F45BC3133008F40E
:1037A000F9C0133009F492C1143029F7109225049E
:1037B000E091D807F0E0EE0FFF1FEB55F84F2081A6
:1037C0003181E091D707F0E0EE0FFF1FEB55F84F86
:1037D000808191813F932F939F938F938EEF93E0FE
:1037E0009F938F9311E01F930E94C30E84E18093F7
:1037F0002504E091DA07F0E0EE0FFF1FEB55F84FDC
:1038000020813181E091D907F0E0EE0FFF1FEB55E9
:10381000F84F808191813F932F939F938F938EEEEA
:1038200093E09F938F931F930E94C30E88E280932F
:103830002504E091DC07F0E0EE0FFF1FEB55F84F99
:1038400020813181E091DB07F0E0EE0FFF1FEB55A7
:10385000F84F808191813F932F939F938F938EEDAB
:1038600093E09F938F931F930E94C30E8CE38093EA
:103870002504E091DE07F0E0EE0FFF1FEB55F84F57
:1038800020813181E091DD07F0E0EE0FFF1FEB5565
:10389000F84F808191813F932F939F938F938EEC6C
:1038A00093E09F938F931F930E94C30E4DB75EB713
:1038B000445E5F4F0FB6F8945EBF0FBE4DBF49C563
:1038C000109226042BCF4093260416CF1092260484
:1038D00020CF1A3009F476C21A3008F4ADC01B307C
:1038E00009F049CF1092250488E192E09F938F93CD
:1038F00011E01F930E94C30E84E180932504209160
:10390000A006332727FD309580919F06992787FDD4
:1039100090953F932F939F938F9388E092E09F938E
:103920008F931F930E94C30E88E2809325042091F9
:10393000A106332727FD30958091A20690E03F93A2
:103940002F939F938F9388EF91E09F938F931F9373
:103950000E94C30E8CE3809325042091A60630E0DC
:103960008091A306992787FD90953F932F939F936E
:103970008F9388EE91E09F938F931F930E94C30EC5
:103980006DB77EB7685E7F4F0FB6F8947EBF0FBEEF
:103990006DBFDFC4112309F4FBC0113009F0EBCE79
:1039A0008091DF0780FF6BC31092250480919E04F5
:1039B00090919F049F938F9387EC94E09F938F93B4
:1039C0001F930E94C30E84E1809325048091A0047C
:1039D0009091A1049F938F9388EB94E09F938F9392
:1039E0001F930E94C30E88E28093250480911803E0
:1039F000909119039F938F9389EA94E09F938F93FB
:103A00001F930E94C30E8CE380932504809190073E
:103A100090E09F938F938AE994E09F938F931F93F5
:103A20000E94C30E4DB75EB74C5E5F4F0FB6F89461
:103A30005EBF0FBE4DBF8DC41092250480918C04D3
:103A400090918D049F938F938EE792E09F938F9335
:103A500011E01F930E94C30E84E18093250480919E
:103A60008E0490918F049F938F9382E792E09F93AF
:103A70008F931F930E94C30E88E280932504809148
:103A80009004909191049F938F9386E692E09F9388
:103A90008F931F930E94C30E8CE380932504809123
:103AA0009204909193049F938F938AE592E09F9361
:103AB0008F931F930E94C30E2DB73EB72C5E3F4FCE
:103AC0000FB6F8943EBF0FBE2DBF43C4109225041D
:103AD0008091A9079091AA072091A7073091A80784
:103AE0009F938F933F932F938EE394E09F938F93B5
:103AF00011E01F930E94C30E84E1809325048091FE
:103B0000AD079091AE072091AB073091AC079F9322
:103B10008F933F932F938EE294E09F938F931F9305
:103B20000E94C30E88E2809325048091B107909192
:103B3000B2072091AF073091B0079F938F933F93C7
:103B40002F938EE194E09F938F931F930E94C30E57
:103B50008CE3809325048091B5079091B60720915E
:103B6000B3073091B4079F938F933F932F938EE0C9
:103B700094E09F938F931F930E94C30E2DB73EB77F
:103B8000245E3F4F0FB6F8943EBF0FBE2DBFE1C37A
:103B90001092250488E095E09F938F9311E01F9386
:103BA0000E94C30E84E18093250420910001822F9E
:103BB0006AE00E94E355492F50E0822F0E94E355AE
:103BC00090E020E730E03F932F9328E430E03F93EC
:103BD0002F931F921F925F934F939F938F9383EF27
:103BE00094E09F938F931F930E94C30E88E280936B
:103BF00025040E94BC0290E09F938F9386EE94E090
:103C00009F938F931F930E94C30E8CE38093250490
:103C100086ED94E09F938F931F930E94C30E2DB760
:103C20003EB7285E3F4F0FB6F8943EBF0FBE2DBF84
:103C300090C384E18093250480910E0390910F033B
:103C40009F938F9385ED92E09F938F9311E01F9345
:103C50000E94C30E88E2809325048091940490E032
:103C60009F938F9386EC92E09F938F931F930E9474
:103C7000C30E6DB77EB7665F7F4F0FB6F8947EBFF9
:103C80000FBE6DBF66C31092250481E193E09F9340
:103C90008F9311E01F930E94C30E84E1809325044B
:103CA0008091390490913A042091060430910704E0
:103CB0009F938F933F932F9382E093E09F938F93F3
:103CC0001F930E94C30E88E28093250480913B04D9
:103CD00090913C0420910404309105049F938F93AC
:103CE0003F932F9383EF92E09F938F931F930E94B4
:103CF000C30E8CE38093250460913F0470914004CF
:103D000080914104909142040E94D954209154081A
:103D1000309155087F936F933F932F9384EE92E0F9
:103D20009F938F931F930E94C30E4DB75EB7485E5B
:103D30005F4F0FB6F8945EBF0FBE4DBF0AC310921F
:103D4000250487EB92E09F938F9311E01F930E94CD
:103D5000C30E84E1809325048091850490918604AC
:103D60009F938F9388EA92E09F938F931F930E9473
:103D7000C30E88E28093250480918104909182048F
:103D80009F938F9389E992E09F938F931F930E9453
:103D9000C30E8CE380932504809183049091840466
:103DA0009F938F938AE892E09F938F931F930E9433
:103DB000C30E8DB79EB742960FB6F8949EBF0FBE46
:103DC0008DBFC7C21092250482E592E09F938F9326
:103DD00011E01F930E94C30E84E18093250480911B
:103DE000AB0390E09F938F9384E492E09F938F9333
:103DF0001F930E94C30E88E2809325048091E903FB
:103E00009091EA039F938F9386E392E09F938F9321
:103E10001F930E94C30E8CE3809325042091FC071E
:103E200030E08091FB0790E03F932F939F938F9317
:103E300088E292E09F938F931F930E94C30E4DB729
:103E40005EB74C5E5F4F0FB6F8945EBF0FBE4DBFBE
:103E500080C2109225048BE794E09F938F9311E02A
:103E60001F930E94C30E84E1809325046091450452
:103E700070914604809147049091480420E034E01A
:103E800040E050E00E9438565F934F933F932F934A
:103E90008CE694E09F938F931F930E94C30E88E259
:103EA0008093250460914D0470914E0480914F04DD
:103EB0009091500420E034E040E050E00E943856F9
:103EC0005F934F933F932F938DE594E09F938F9350
:103ED0001F930E94C30E8CE380932504809181047C
:103EE000909182049F938F938EE494E09F938F939D
:103EF0001F930E94C30E8DB79EB746960FB6F894D7
:103F00009EBF0FBE8DBF25C21092250480EC93E0AA
:103F10009F938F9311E01F930E94C30E8091000125
:103F20000F900F900F908A3009F471C18B3009F413
:103F3000C4C0843109F4C1C08D3009F00AC284E1E3
:103F40008093250480911A0390E020912F043091F2
:103F50003004A90137FDFAC1BA01759567957595C9
:103F6000679575956795759567954091FE03509196
:103F7000FF0337FDE8C1359527953595279535958C
:103F80002795421B530B9F938F937F936F935F9360
:103F90004F9386E493E09F938F931F930E94C30EE9
:103FA00088E28093250480911B0390E020913104E6
:103FB00030913204A9016DB77EB7675F7F4F0FB6AE
:103FC000F8947EBF0FBE6DBF37FDBAC1BA017595BB
:103FD0006795759567957595679575956795409102
:103FE00000045091010437FDA8C1359527953595FA
:103FF000279535952795421B530B9F938F937F935E
:104000006F935F934F9382E393E09F938F931F93FC
:104010000E94C30E8CE38093250480911C03682FBB
:1040200070E02091330430913404A9018DB79EB71C
:1040300009960FB6F8949EBF0FBE8DBF37FD7AC1AB
:10404000559547958091020490910304281B390BE4
:104050007F936F935F934F933F932F938EE193E002
:104060009F938F931F930E94C30E2DB73EB7275F78
:104070003F4F0FB6F8943EBF0FBE2DBF6AC184E11B
:104080008093250483E994E09F938F931F930E946C
:10409000C30E88E28093250485E894E09F938F9374
:1040A0001F930E94C30E6DB77EB76A5F7F4F0FB636
:1040B000F8947EBF0FBE6DBF4CC184E18093250490
:1040C000E0912F04F0913004CF0160E170E00E9494
:1040D000035697FD27C1BC01759567959F01F7FDB4
:1040E0001EC1A901559547955595479555954795F5
:1040F000559547952091FE033091FF03CF01F7FDC1
:104100000CC1959587959595879595958795281BCD
:10411000390B7F936F935F934F933F932F938BE76D
:1041200093E09F938F931F930E94C30E88E2809326
:104130002504E0913104F0913204CF0160E170E098
:104140000E9403562DB73EB7275F3F4F0FB6F89436
:104150003EBF0FBE2DBF97FDDEC0BC0175956795B4
:104160009F01F7FDD5C0A9015595479555954795F0
:104170005595479555954795209100043091010438
:10418000CF01F7FDC3C09595879595958795959532
:104190008795281B390B7F936F935F934F933F93C2
:1041A0002F9389E693E09F938F931F930E94C30EF2
:1041B0008CE3809325042091330430913404A901C9
:1041C0006DB77EB7675F7F4F0FB6F8947EBF0FBEA7
:1041D0006DBF37FD98C05595479580910204909129
:1041E0000304281B390B5F934F933F932F938AE56A
:1041F00093E09F938F931F930E94C30E8DB79EB73A
:1042000007960FB6F8949EBF0FBE8DBFA2C084E183
:104210008093250420912F0430913004C90168E077
:1042200070E00E940356AC0137FD81C0359527959B
:1042300035952795359527958091FE039091FF033D
:10424000821B930B5F934F933F932F939F938F9377
:104250008EEA93E09F938F931F930E94C30E88E290
:10426000809325042091310430913204C90168E023
:1042700070E00E940356AC016DB77EB7675F7F4F59
:104280000FB6F8947EBF0FBE6DBF37FD4DC035959C
:104290002795359527953595279580910004909120
:1042A0000104821B930B5F934F933F932F939F9334
:1042B0008F938CE993E09F938F931F930E94C30E7B
:1042C0008CE3809325042091330430913404809151
:1042D000020490910304A901481B590B3F932F93AB
:1042E0005F934F938DE893E09F938F931F930E946A
:1042F000C30E6DB77EB7605F7F4F0FB6F8947EBF79
:104300000FBE6DBF26C04F5F5F4F65CF07963BCF97
:10431000215F3F4F28CF019620CF0796F2CE215F35
:104320003F4FDFCE0196D7CE295F3F4FB0CF295FF9
:104330003F4F7CCF4F5F5F4F83CE295F3F4F55CEBE
:10434000415F5F4F43CE295F3F4F15CE415F5F4FC7
:1043500003CE109227041F9108951092B9008AE2AB
:104360008093B800089585EA8093BC0080E090E0D7
:10437000089584E98093BC0008951092B900809359
:10438000BB0085E88093BC0080E090E008950E9427
:10439000B92110922804EBEBF0E0808110922904FF
:1043A00080E88093BC001092BD001092BA00108289
:1043B0001092B9001092B8000E94AD210E94B32162
:1043C00080E00E94BD2108951F920F920FB60F92B8
:1043D00011242F933F934F935F936F937F938F930A
:1043E0009F93AF93BF93EF93FF93809128048F5FC8
:1043F000809328048150E82FF0E0E731F10508F0C0
:10440000ABC0E05BFF4FEE0FFF1F0590F491E02D76
:1044100009948091BB0090912A04E92FF0E0EB56BB
:10442000F84F8083913009F46EC0913008F487C052
:10443000923009F489C0933009F08EC080916E08E3
:104440000E94BD2189C088E90E94BD2185C080E805
:104450000E94BD2181C00E94B9218AE090E0909322
:104460009403809393030E94B32176C090912A0411
:104470008091BB00E92FF0E0EB56F84F84839F5FFB
:1044800090932A04943010F010922A040E94B921CB
:104490008AE090E090939403809393031092280411
:1044A0005BC00E94B92180912904843008F051C07A
:1044B00010922804D8CF80911C030E94BD214CC0CB
:1044C00080911A030E94BD2147C080912904880F62
:1044D0008E5A0E94BD2140C080E10E94BD213CC097
:1044E00080912A04813079F0813048F1823061F185
:1044F000833091F5A3CF809129048F5F80932904A5
:104500008150813089F7809145080E94BD2124C0E7
:1045100084E10E94BD2120C080911B030E94BD2127
:104520001BC082E10E94BD2117C080912A04880F20
:104530008D5A0E94BD2110C090912A0473CF8091A2
:1045400038080E94BD2108C0809169080E94BD21E1
:1045500003C01092290487CF8091BC0080688093AB
:10456000BC00FF91EF91BF91AF919F918F917F918F
:104570006F915F914F913F912F910F900FBE0F90D0
:104580001F90189583EC80938100EFE6F0E0808126
:1045900080628083109234041092330410923204AB
:1045A000109231041092300410922F0408951F923B
:1045B0000F920FB60F9211240F931F932F933F93D7
:1045C0004F935F936F937F938F939F93AF93BF931B
:1045D000CF93DF93EF93FF93209186003091870074
:1045E00080912D0490912E04281B390B8091860018
:1045F0009091870090932E0480932D04C9018D54CF
:104600009440835F9A4170F480912B0490912C0424
:1046100004970CF07EC081E090E090932C0480938E
:104620002B049DC000912B0410912C040A3011051D
:104630000CF095C0C9018B5F9040845B914008F0FD
:1046400056C0A901425D5140E801CC0FDD1FFE01BB
:10465000EB55F84F808191819A01281B390BC901D4
:1046600037FD79C0069754F480919404883C08F093
:104670006BC080919404865F80939404FE01EB5597
:10468000F84F808191819C01220F331F280F391F21
:10469000240F351F37FD5CC0359527953595279537
:1046A000CA010196821793070CF045C02150304093
:1046B00080919404833CC8F1FE01EB55F84F808152
:1046C0009181A901481B590BCA0163E070E00E9467
:1046D0000356CB01880F991F860F971FFE01E554E3
:1046E000F84F91838083CB55D84F39832883C801F5
:1046F000019690932C0480932B048530910589F0CA
:104700005D988630910551F05C98079729F05B9889
:1047100026C0109279037FCF5B9A21C05C9A5B9888
:104720001EC05D9A5C985B981AC0FE01E554F84F74
:1047300011821082D8CF41505040241735070CF019
:10474000B7CF2F5F3F4FB4CF88EC8093940496CFC0
:104750002D5F3F4FA1CF909581959F4F83CFFF91C4
:10476000EF91DF91CF91BF91AF919F918F917F9109
:104770006F915F914F913F912F911F910F910F90EA
:104780000FBE0F901F90189581E08093D70782E0AD
:104790008093D80783E08093D90784E08093DA0779
:1047A00085E08093DB0786E08093DC0787E08093D9
:1047B000DD0788E08093DE0708956817790744F4E1
:1047C000680F791F77FD09C0CB01959587950895EE
:1047D000681B790B861B970B08956F5F7F4FCB018A
:1047E0009595879508952F923F924F925F926F9281
:1047F0007F928F929F92AF92BF92CF92DF92EF9271
:10480000FF920F931F93CF93DF93CDB7DEB76B97D4
:104810000FB6F894DEBF0FBECDBF80910204909119
:1048200003044090330450903404481A590A5092BB
:104830007808409277082091F8033091F90337FF08
:1048400002C00C94112C35952795359527953595F3
:1048500027953B8F2A8F2091FA033091FB0337FD78
:10486000DDC73595279535952795359527953C8B4B
:104870002B8B2A8D3B8D30935708209356088B89BC
:104880009C8990934B0880934A086091060470912C
:104890000704882777FD8095982F26E030E040E0D8
:1048A00050E00E94C4557B018C0120917208309128
:1048B0007308442737FD4095542FCA01B901660F8C
:1048C000771F881F991F620F731F841F951F6E0D1E
:1048D0007F1D801F911F24E030E040E050E00E94E7
:1048E00038563093730820937208609104047091D5
:1048F0000504882777FD8095982F26E030E040E07A
:1049000050E00E94C4557B018C01209182083091B7
:104910008308442737FD4095542FCA01B901660F1B
:10492000771F881F991F620F731F841F951F6E0DBD
:104930007F1D801F911F24E030E040E050E00E9486
:1049400038563093830820938208E0900804F09052
:1049500009042091540830915508442737FD4095AB
:10496000542FCA01B901660F771F881F991F620F64
:10497000731F841F951F0027F7FC0095102F6E0DE5
:104980007F1D801F911F24E030E040E050E00E9436
:1049900038563093550820935408209106043091DE
:1049A0000704C901880F991F820F931F880F991F51
:1049B000AA2797FDA095BA2F20915504309156044F
:1049C0004091570450915804280F391F4A1F5B1F0C
:1049D0002093550430935604409357045093580441
:1049E0002091040430910504C901880F991F820F9A
:1049F000931F880F991FAA2797FDA095BA2F209182
:104A0000590430915A0440915B0450915C04280F82
:104A1000391F4A1F5B1F2093590430935A04409357
:104A20005B0450935C04209106043091070480914C
:104A30005F0890916008820F931F909360088093A5
:104A40005F08209104043091050480917A089091C8
:104A50007B08820F931F90937B0880937A08809144
:104A60003D0490913E04019690933E0480933D0452
:104A7000E0908507F0908607A0903F04B090400436
:104A8000C0904104D090420460915D0470915E0436
:104A900080915F04909160040E940C553B014C0191
:104AA0000027F7FC0095102FC801B7010E940C5594
:104AB000A60195010E9474549B01AC01C401B3018D
:104AC0000E9475540E94D95460935D0470935E04F3
:104AD00080935F04909360048FEC80937A0010922F
:104AE0001D0380916D0490916E04A0916F04B091AC
:104AF00070048F87988BA98BBA8B809165049091F5
:104B00006604A0916704B09168048B879C87AD8789
:104B1000BE873201882477FC8094982C809175049C
:104B200090917604A0917704B0917804860D971D3A
:104B3000A81DB91D8E8B9F8BA88FB98F809375048C
:104B400090937604A0937704B093780420907E0825
:104B500030907F084090800850908108260C371CC8
:104B6000481C591C20927E0830927F084092800891
:104B7000509281089091A6049A87992329F48091F4
:104B8000A704882309F474C4A091DF07A9831092B5
:104B9000D6071092D5071092D2071092D107109223
:104BA00018051092190510921A0510921B05109203
:104BB0001C0510921D0510921E0510921F05B09144
:104BC000AF03BD8BE0901C05F0901D0500911E0504
:104BD00010911F05A0901805B0901905C0901A05F6
:104BE000D0901B05C601B50124E630E040E050E05E
:104BF0000E9438564701821A930A90924408809284
:104C00004308C801B70124E630E040E050E00E94CC
:104C1000385639016A187B0870923A086092390850
:104C20006091B3037091B4038091B5039091B60382
:104C300028E631E040E050E00E94C45526163706D1
:104C40004806590664F0261A370A480A590A20927B
:104C50007E0830927F08409280085092810857FC6D
:104C600056C56B897C89680D791D9B01442737FDEA
:104C70004095542F8091710490917204A091730417
:104C8000B0917404820F931FA41FB51F8093710409
:104C900090937204A0937304B09374048091A2045F
:104CA0009091A304681B790B7B010027F7FC00950A
:104CB000102F8F859889A989BA89E80EF91E0A1FD5
:104CC0001B1FE0926D04F0926E0400936F0410932A
:104CD000700420919B0330919C0340919D0350915F
:104CE0009E032E153F0540075107D4F478EAE72EBE
:104CF00071E6F72E012D112DE21AF30A040B150BA4
:104D0000E0926D04F0926E0400936F0410937004AF
:104D1000E0927104F092720400937304109374048F
:104D200088279927DC01821B930BA40BB50BE0901D
:104D30006D04F0906E0400916F0410917004E816F9
:104D4000F9060A071B07E4F468E5E62E6EE9F62E7D
:104D50006FEF062F6FEF162FE20EF31E041F151FC5
:104D6000E0926D04F0926E0400936F04109370044F
:104D7000E0927104F092720400937304109374042F
:104D80006A8D7B8D660D771D9B01442737FD40950D
:104D9000542F8091690490916A04A0916B04B091A2
:104DA0006C04820F931FA41FB51F80936904909316
:104DB0006A04A0936B04B0936C048091A404909156
:104DC000A504681B790B9B01442737FD4095542FA0
:104DD0008B859C85AD85BE85280F391F4A1F5B1FBB
:104DE00020936504309366044093670450936804ED
:104DF000A0909703B0909803C0909903D0909A0325
:104E0000A216B306C406D506C4F428EA31E640E08B
:104E100050E02A193B094C095D0920936504309341
:104E200066044093670450936804209369043093A8
:104E30006A0440936B0450936C0488279927DC0123
:104E40008A199B09AC09BD0920916504309166045B
:104E50004091670450916804281739074A075B0797
:104E6000B4F4A6019501285A3146404050402093A1
:104E7000650430936604409367045093680420935C
:104E8000690430936A0440936B0450936C048E89D8
:104E90009F89A88DB98D8093610490936204A0933B
:104EA0006304B09364042093450430934604409314
:104EB000470450934804E0924D04F0924E0400934E
:104EC0004F04109350048091690490916A04A0915A
:104ED0006B04B0916C048093490490934A04A093AE
:104EE0004B04B0934C048091710490917204A09192
:104EF0007304B09174048093510490935204A0936E
:104F00005304B0935404809110039091110397FDC2
:104F1000FCC39595879595958795959587959093DD
:104F2000470880934608809112039091130397FDE0
:104F300073C4959587959595879595958795909345
:104F40003708809336088091FE039091FF030F97F6
:104F500034F488E19CEF9093470880934608809151
:104F6000FE039091FF03079734F480E398EF90934A
:104F7000470880934608209100012A3009F4DAC1DD
:104F80008091FE039091FF03815D974034F088EE9D
:104F900093E090934708809346088091FE03909198
:104FA000FF03805E97400CF0DAC18091000490917D
:104FB00001040F9734F488E19CEF909337088093B5
:104FC00036088091000490910104079734F480E33F
:104FD00098EF90933708809336082A3009F48EC1F1
:104FE0008091000490910104815D974034F088EE37
:104FF00093E0909337088093360880910004909155
:105000000104805E97400CF08EC16091A603662378
:1050100009F4A2C0409110035091110380910E0534
:1050200090910F05481B590B5093090540930805B3
:105030002091100330911103280F391F37FDF5C35C
:105040003595279530930F0520930E05413851056E
:105050000CF403C280E890E0909309058093080562
:10506000E62FF0E08091080590910905E89FB001D6
:10507000E99F700DF89F700D11249B0177FDE0C32F
:105080003595279535952795359527953595279508
:105090008091460890914708820F931F909347088C
:1050A00080934608409112035091130380910C05A0
:1050B00090910D05481B590B50930B0540930A0521
:1050C0002091120330911303280F391F37FDBEC3FF
:1050D0003595279530930D0520930C0541385105E2
:1050E0000CF408C380E890E090930B0580930A05C8
:1050F00080910A0590910B05E89FA001E99F500D52
:10510000F89F500D11249A0157FD9DC335952795A1
:1051100035952795359527953595279580913608AE
:1051200090913708820F931F909337088093360829
:105130008091100390911103680F791F70931103F0
:10514000609310038091120390911303480F591F2D
:1051500050931303409312038B899C8918161906E8
:105160000CF0E2C29D89E92EFF2400E010E060917E
:10517000D1077091D20777FD5FC3882777FD8095AF
:10518000982FA80197010E94C45520E430E040E028
:1051900050E00E943856820E931E909244088092EE
:1051A0004308EA8DFB8D1E161F060CF0E2C220910B
:1051B000D5073091D60737FD3BC3442737FD4095CF
:1051C000542FC801B7010E94C45520E430E040E0EC
:1051D00050E00E943856620E731E70923A08609238
:1051E0003908F981F7FDE2C28091DB07E82FF0E092
:1051F000EE0FFF1FEB55F84F80819181A0918C0439
:10520000B0918D0482599F4FA817B9070CF0FFC0C9
:105210001196B0938D04A0938C048091DC07E82F45
:10522000F0E0EE0FFF1FEB55F84F80819181609108
:105230008E0470918F0482599F4F681779070CF084
:10524000D3C06F5F7F4F70938F0460938E04809103
:10525000DD07E82FF0E0EE0FFF1FEB55F84F8081E0
:105260009181409190045091910482599F4F481729
:1052700059070CF0A6C04F5F5F4F509391044093C5
:1052800090048091DE07E82FF0E0EE0FFF1FEB5552
:10529000F84F80819181209192043091930482593A
:1052A0009F4F281739070CF061C02F5F3F4F309395
:1052B000930420939204B7FD6DC0AF3FB10511F088
:1052C0000CF0C4C077FD6CC06F3F710511F00CF09D
:1052D000B6C057FD6BC04F3F510511F00CF0A8C090
:1052E00037FD6AC02F3F310509F00CF4EEC28FEF95
:1052F00090E09093930480939204E7C2809100041D
:1053000090910104835F934034F088EE93E0909392
:1053100037088093360880910004909101048A5FD9
:1053200093400CF472CE80ED97E090933708809311
:1053300036086BCE8091FE039091FF03835F93400C
:1053400034F088EE93E0909347088093460880916C
:10535000FE039091FF038A5F93400CF426CE80ED0C
:1053600097E090934708809346081FCE80819181F3
:1053700082599F4F821793070CF09DCF211531055D
:1053800009F499CF21503040309393042093920434
:10539000B7FF93CF10928D0410928C0477FF94CFB7
:1053A00010928F0410928E0457FF95CF10929104A3
:1053B0001092900437FF96CF1092930410929204AB
:1053C00084C28081918182599F4F841795070CF088
:1053D00058CF4115510509F454CF415050405093D6
:1053E0009104409390044DCF8081918182599F4FC9
:1053F000861797070CF02BCF6115710509F427CF9D
:105400006150704070938F0460938E0420CF808130
:10541000918182599F4F8A179B070CF0FECE1097FF
:1054200009F4FBCE1197B0938D04A0938C04F5CEB4
:105430008FEF90E0909391048093900451CF8FEF81
:1054400090E090938F0480938E0443CF8FEF90E091
:1054500090938D0480938C0435CF40585F4F0CF0AF
:10546000FFCD80E89FEF9093090580930805F8CD64
:10547000B091DF07B983B6FF8ACB2F853889498978
:105480005A89283BE4E93E07EEEF4E07EFEF5E074F
:1054900024F428EB34E94EEF5FEF2A833B834C83FF
:1054A0005D8329543B464140504044F088E49BE6EC
:1054B000A1E0B0E08A839B83AC83BD832B853C85D0
:1054C0004D855E85283B94E939079EEF49079FEF9C
:1054D000590724F428EB34E94EEF5FEF2E833F8326
:1054E0004887598729543B464140504044F088E45E
:1054F0009BE6A1E0B0E08E839F83A887B987A09048
:10550000AE03BB24CC24DD24AB89BC899D01442798
:1055100037FD4095542F6E817F81888599850E9443
:10552000C45520E038E040E050E00E943856CA01FF
:10553000B901A60195010E94C45520E030E140E088
:1055400050E00E94385679018A0120931405309367
:1055500015054093160550931705EA8DFB8D9F01A5
:10556000442737FD4095542F6A817B818C819D8132
:105570000E94C45520E038E040E050E00E943856D8
:10558000CA01B901A60195010E94C45520E030E18D
:1055900040E050E00E943856F092D207E092D107E6
:1055A0003093D6072093D5072E193F09400B510B96
:1055B00079018A012093100530931105409312055B
:1055C00050931305220E331E441E551E20927E0852
:1055D00030927F084092800850928108F091AF038A
:1055E000FD8BFF23E1F4CA01B90122E030E040E085
:1055F00050E00E9438568E899F89A88DB98D821BF4
:10560000930BA40BB50B8E8B9F8BA88FB98F8093B8
:10561000750490937604A0937704B09378046E0C8D
:105620007F1C801E911EE090AD03FF2400E010E07F
:10563000C401B3012E813F81488559850E94C4551C
:1056400020E038E040E050E00E943856CA01B9013D
:10565000A80197010E94C45520E030E140E050E0ED
:105660000E94385659016A0120931C0530931D058C
:1056700040931E0550931F05C401B3012A813B814D
:105680004C815D810E94C45520E038E040E050E04C
:105690000E943856CA01B901A80197010E94C45559
:1056A00020E030E140E050E00E9438562093180599
:1056B0003093190540931A0550931B05D7FCE8C099
:1056C00091E8A916B104C104D10444F457FDD8C02F
:1056D00021383105410551050CF474CA81E08093ED
:1056E000890420907E0830907F0840908008509078
:1056F000810868CA40585F4F0CF0FACC80E89FEFF1
:1057000090930B0580930A05F3CC079602CC260EE6
:10571000371E481E591E20927E0830927F08409204
:105720008008509281089DCAAD89EA2EFF2400E0CE
:1057300010E06091D1077091D20777FD8AC0882769
:1057400077FD8095982FA80197010E94C45520E409
:1057500030E040E050E00E943856821A930A90925E
:10576000440880924308EA8DFB8D1E161F060CF438
:105770001ECD2091D5073091D60737FD6EC0442746
:1057800037FD4095542FC801B7010E94C45520E44D
:1057900030E040E050E00E943856621A730A70927E
:1057A0003A0860923908F981F7FF1ECD2A85222335
:1057B00009F01ACD8091A704882309F015CD8A8DB0
:1057C0009B8D815091400CF04CC02A8D3B8D6FEF2A
:1057D0002030360764F48091460890914708805045
:1057E0009F4F820F931F90934708809346088B89A1
:1057F0009C89815091400CF454C08091360890915E
:10580000370880509140EB89FC898E0F9F1F909341
:10581000370880933608E8CC07968BCB295F3F4F3B
:1058200020C8295F3F4F0C9423242F5F3F4F08CCA3
:10583000309521953F4FC1CC709561957F4F9DCCA0
:10584000215F3F4F1DCC215F3F4F60CC2F5F3F4F0B
:105850003FCC709561957F4F72CF309521953F4F2A
:105860008ECF809146089091470880509140EA8DF4
:10587000FB8D8E0F9F1F9093470880934608B7CFEC
:1058800050954095309521953F4F4F4F5F4F20CF1A
:10589000D094C094B094A094A11CB11CC11CD11C84
:1058A0000FCF2B893C896FEF203036070CF09CCC52
:1058B000809136089091370880509F4F820F931F38
:1058C00090933708809336088FCC6B960FB6F89478
:1058D000DEBF0FBECDBFDF91CF911F910F91FF9023
:1058E000EF90DF90CF90BF90AF909F908F907F9080
:1058F0006F905F904F903F902F9008958091E207B6
:105900008B3F80F08B3F09F407C38C3F09F4D6C36B
:105910008D3F09F43DC38E3F39F48091920480930A
:10592000A20302C08093A2038091E1078B3F80F025
:105930008B3F09F4F6C28C3F09F4C5C38D3F09F4CF
:105940002CC38E3F39F4809192048093A10302C04E
:105950008093A1038091A1038823B1F41092A10345
:105960008091E3078B3FC8F08B3F09F4E4C28C3F82
:1059700009F4AEC38D3F09F415C38E3F81F48091C5
:1059800092048093A3030BC0843650F384E6809383
:10599000A1038091E3078B3F38F78093A3038091A5
:1059A000A3038823B1F41092A3038091E5078B3FF2
:1059B000C8F08B3F09F4BAC28C3F09F4CAC38D3FCB
:1059C00009F4E1C28E3F81F4809192048093A40394
:1059D0000BC0843650F384E68093A3038091E507DF
:1059E0008B3F38F78093A4038091EC078B3F80F0C6
:1059F0008B3F09F47DC28C3F09F4A6C38D3F09F4A7
:105A0000BDC28E3F39F4809192048093A50302C0F9
:105A10008093A5038091ED078B3F80F08B3F09F4C5
:105A20006CC28C3F09F481C38D3F09F498C28E3F4C
:105A300039F4809192048093A70302C08093A70356
:105A40008091A7038B30B8F48AE08093A7038091FC
:105A5000EE078B3FC0F08B3F09F454C28C3F09F432
:105A600069C38D3F09F480C28E3F79F4809192041E
:105A70008093A8030AC08F3F51F78093A7038091BA
:105A8000EE078B3F40F78093A8038091EF078B3F91
:105A900080F08B3F09F41DC28C3F09F450C38D3F49
:105AA00009F467C28E3F39F4809192048093A60373
:105AB00002C08093A6038091F4078B3F80F08B3F58
:105AC00009F425C28C3F09F4D1C28D3F09F488C284
:105AD0008E3F39F4809192048093AA0302C0809390
:105AE000AA038091F5078B3F80F08B3F09F4F6C144
:105AF0008C3F09F4C0C28D3F09F477C28E3F39F460
:105B0000809192048093AC0402C08093AC04809195
:105B1000F6078B3F80F08B3F09F4E5C18C3F09F419
:105B2000AFC28D3F09F466C28E3F39F48091920472
:105B30008093AD0402C08093AD048091F7078B3F42
:105B400080F08B3F09F4BBC18C3F09F4DAC28D3F72
:105B500009F441C28E3F39F4809192048093AE04DF
:105B600002C08093AE048091F8078B3F80F08B3F9A
:105B700009F4AAC18C3F09F46AC28D3F09F462C2DC
:105B80008E3F39F4809192048093AF0402C08093D9
:105B9000AF04809109088B3F80F08B3F09F485C1E9
:105BA0008C3F09F486C28D3F09F43DC28E3F39F423
:105BB000809192048093B00402C08093B0048091DD
:105BC0000A088B3F80F08B3F09F474C18C3F09F4C5
:105BD00043C28D3F09F42CC28E3F39F48091920468
:105BE0008093B10402C08093B10480910B088B3F75
:105BF00080F08B3F09F44FC18C3F09F432C28D3FD6
:105C000009F41BC28E3F39F4809192048093B20450
:105C100002C08093B20480910C088B3F80F08B3FD0
:105C200009F43EC18C3F09F435C28D3F09F4ECC143
:105C30008E3F39F4809192048093B30402C0809324
:105C4000B3048091F9078B3F80F08B3F09F419C1B1
:105C50008C3F09F424C28D3F09F4DBC18E3F39F437
:105C6000809192048093AB0302C08093AB03809138
:105C7000FE078B3F80F08B3F09F408C18C3F09F48D
:105C800013C28D3F09F4CAC18E3F39F4809192044A
:105C90008093AC0302C08093AC03809101088B3FDA
:105CA00080F08B3F09F4E3C08C3F09F4EEC18D3FD7
:105CB00009F4A5C18E3F39F4809192048093AD031D
:105CC00002C08093AD03809102088B3F80F08B3F30
:105CD00009F4D2C08C3F09F40FC28D3F09F476C19C
:105CE0008E3F39F4809192048093AE0302C080937A
:105CF000AE03809103088B3F80F08B3F09F4ADC069
:105D00008C3F09F4EAC18D3F09F451C18E3F39F44B
:105D1000809192048093AF0302C08093AF0380917F
:105D200008088B3F80F08B3F09F49CC08C3F09F43E
:105D3000D9C18D3F09F440C18E3F39F4809192045E
:105D40008093B00302C08093B00380910E088B3F14
:105D500080F08B3F09F47CC08C3F09F4C8C18D3FB3
:105D600009F42FC18E3F39F4809192048093610829
:105D700002C08093610880916108823008F455C0A8
:105D80008F3F09F448C0809110088B3F80F08B3F13
:105D900009F44FC08C3F09F4B9C18D3F09F4D0C05C
:105DA0008E3F39F4809192048093750802C08093ED
:105DB0007508809175088230A0F18F3F79F180914C
:105DC00011088B3F78F08B3FF1F18C3F09F4A3C1B0
:105DD0008D3F09F4BAC08E3F39F4809192048093CC
:105DE000420802C080934208809121088B3F80F0D6
:105DF0008B3F21F18C3F09F493C18D3F09F4AAC078
:105E00008E3F09F0ABC18091920480938608A6C1B1
:105E100080938608A3C180936108B5CF80937508ED
:105E2000CECF81E080937508CACF81E0809361086E
:105E3000AACF80918C0480937508BBCF80918C048D
:105E4000809386088BC180918C0480934208CCCFCC
:105E500080918C04809361088ECF80918C04809314
:105E6000AF035DCF80918C048093B0036ECF80919F
:105E70008C048093AD0327CF80918C048093AE0374
:105E800038CF80918C048093AB03F1CE80918C0449
:105E90008093AC0302CF80918C048093B204BBCE7C
:105EA00080918C048093B304CCCE80918C04809339
:105EB000B00485CE80918C048093B10496CE8091FD
:105EC0008C048093AE044FCE80918C048093AF04F9
:105ED00060CE80918C048093A603EDCD80918C04DC
:105EE0008093AC0414CE80918C048093AD0425CEB5
:105EF00080918C048093A5038DCD80918C04809338
:105F0000A7039ECD80918C048093A803BECD809181
:105F10008C048093AA03E5CD80918C048093A20326
:105F200003CD80918C048093A10314CD80918C04C7
:105F30008093A40359CD80918C048093A3032FCD2B
:105F4000809190048093750834CF80919004809361
:105F500042084ACF8091900480938608FFC08091C8
:105F600090048093A7036CCD809190048093A80344
:105F70008CCD809190048093A6039DCD8091900458
:105F80008093A50347CD809190048093A4032CCDEA
:105F9000809190048093A203C7CC80919004809359
:105FA000A103D8CC809190048093A303F8CC809176
:105FB00090048093AF03B3CE809190048093B0039C
:105FC000C4CE8091900480936108D5CE80919004D6
:105FD0008093AE038ECE809190048093AE04C3CDA7
:105FE000809190048093AA037CCD8091900480934B
:105FF000AC048DCD809190048093AD049ECD8091B2
:1060000090048093AD035FCE809190048093B3049D
:1060100018CE809190048093AB0329CE8091900498
:106020008093AC033ACE809190048093B004C7CDA6
:10603000809190048093B104D8CD80919004809396
:10604000B204E9CD809190048093AF04A2CD8091F9
:106050008E048093AF049DCD80918E048093B10413
:10606000C4CD80918E048093B204D5CD80918E04EE
:106070008093AA0336CD80918E048093AC0447CDE3
:1060800080918E048093AD0458CD80918E048093CE
:10609000AD0319CE80918E048093B304D2CD80914C
:1060A0008E048093AB03E3CD80918E048093AC0388
:1060B000F4CD80918E048093B00481CD80918E04C4
:1060C0008093A20331CC80918E048093A10342CCB3
:1060D00080918E048093A30362CC80918E04809380
:1060E000AF031DCE80918E048093B0032ECE80919D
:1060F0008E04809361083FCE80918E048093AE031E
:10610000F8CD80918E048093AE042DCD80918E04C5
:10611000809375084ECE80918E048093420864CEA1
:1061200080918E048093860819C080918E0480939C
:10613000A70386CC80918E048093A803A6CC80917F
:106140008E048093A603B7CC80918E048093A50320
:1061500061CC80918E048093A40346CC6091AA0305
:1061600070E06F5F7F4F8CE398E20E94035670935C
:10617000A00360939F038091EA0780937608809143
:10618000E90780934C08089580919D04882321F5A8
:1061900010924508109238081092690810926E0803
:1061A0008091D203882311F0809338088091D30323
:1061B000882311F0809345088091D403882311F03F
:1061C00080936E088091D503882361F48091C00488
:1061D0008C7F8093C00409C08091C004816080934B
:1061E000C00403C080936908F1CF8091380890E023
:1061F00090935A07809359078091450890E09093B7
:106200005C0780935B0780916E0890E090935E0737
:1062100080935D078091690890E090936007809378
:106220005F0710922804109229040E94B321089558
:10623000809100018D3009F443C110927A00809161
:10624000FE039091FF039093470880934608809146
:106250000004909101049093370880933608809150
:1062600002049091030490937808809377086091DA
:10627000060470910704882777FD8095982F26E003
:1062800030E040E050E00E94C45570937308609382
:1062900072086091040470910504882777FD809549
:1062A000982F0E94C4557093830860938208809150
:1062B00008049091090490935508809354088FEC3A
:1062C00080937A008091DB07E82FF0E0EE0FFF1F4C
:1062D000EB55F84F80819181A0918C04B0918D0491
:1062E00082599F4FA817B9070CF0C4C01196B093FC
:1062F0008D04A0938C048091DC07E82FF0E0EE0F72
:10630000FF1FEB55F84F8081918160918E04709151
:106310008F0482599F4F681779070CF098C06F5F00
:106320007F4F70938F0460938E048091DD07E82F78
:10633000F0E0EE0FFF1FEB55F84F80819181409107
:1063400090045091910482599F4F481759070CF0BF
:106350006BC04F5F5F4F50939104409390048091C6
:10636000DE07E82FF0E0EE0FFF1FEB55F84F8081BE
:106370009181209192043091930482599F4F281764
:1063800039074CF52F5F3F4F3093930420939204CD
:10639000B7FD33C0AF3FB10511F00CF08AC077FDF7
:1063A00032C06F3F710511F00CF07CC057FD31C059
:1063B0004F3F510511F00CF06EC037FD30C02F3F3C
:1063C000310509F00CF47FC08FEF90E090939304B7
:1063D0008093920478C08081918182599F4F821767
:1063E0009307B4F62115310599F2215030403093CE
:1063F000930420939204B7FFCDCF10928D04109296
:106400008C0477FFCECF10928F0410928E0457FF2A
:10641000CFCF109291041092900437FFD0CF1092FA
:106420009304109292044FC08081918182599F4FB2
:10643000841795070CF093CF4115510509F48FCFC0
:1064400041505040509391044093900488CF8081F4
:10645000918182599F4F861797070CF066CF61157F
:10646000710509F462CF6150704070938F0460939E
:106470008E045BCF8081918182599F4F8A179B0741
:106480000CF039CF109709F436CF1197B0938D04E3
:10649000A0938C0430CF8FEF90E090939104809381
:1064A00090048BCF8FEF90E090938F0480938E04B5
:1064B0007DCF8FEF90E090938D0480938C046FCF0D
:1064C0000E94351ABACE6091040870E080E090E036
:1064D00024EC39E040E050E00E94C45560939703FB
:1064E000709398038093990390939A0360910508A1
:1064F00070E080E090E00E94C45560939B0370932D
:106500009C0380939D0390939E0308956F927F92C6
:106510008F929F92AF92BF92CF92DF92EF92FF92B3
:106520000F931F93CF93DF931092E803469A109234
:106530003A041092390410923C0410923B0480E01B
:1065400090E0A0E0B0E080933F0490934004A093DB
:106550004104B09342041092300410922F04109220
:1065600032041092310410923404109233041092C9
:106570006708109266081092AD031092AE03109255
:106580000B040E94183184E690E00E94A7120E943A
:1065900018318091DF0780FF10C08091180390911F
:1065A0001903875B934008F0D8C08091180390913D
:1065B00019038E5E924008F4D0C0EE24CC24DD2472
:1065C000C0E0D0E000E010E08AE090E00E94A71276
:1065D0008091020490910304C80ED91E8091FE039D
:1065E0009091FF03C80FD91F80910004909101047E
:1065F000080F191FE39480E2E81631F7AE01405FFF
:106600005F4F569547955695479550933004409364
:106610002F049801205F3F4F369527953695279593
:106620003093320420933104C601409696958795A5
:10663000929582958F7089279F7089279093340453
:1066400080933304909367088093660830933604F0
:1066500020933504509338044093370444E050E0CD
:10666000DA010E945356802D853078F1809182089E
:106670009091830897FD78C06CE070E00E9403560B
:1066800070933C0460933B0480917208909173086E
:1066900097FD66C06CE070E00E94035670933A0468
:1066A000609339046091850770918607882777FD8C
:1066B0008095982F0E940C5560933F04709340047E
:1066C000809341049093420453C0DA010E945356D0
:1066D000802D4F5F5F4FDA010E945356202D90E0CE
:1066E000982F8827820F911D90933A048093390444
:1066F0004F5F5F4FDA010E945356802D4F5F5F4F0F
:10670000DA010E945356202D90E0982F8827820F9F
:10671000911D90933C0480933B044F5F5F4FDA01DF
:106720000E945356602D4F5F5F4FDA010E9453560F
:10673000202D70E0762F6627620F711D882777FD68
:106740008095982F0E940C5560933F0470934004ED
:1067500080934104909342040BC00E94FC1A2DCFF9
:10676000909581959F4F96CF909581959F4F84CF1F
:106770001092470810924608109237081092360877
:10678000109278081092770884E690E00E94A71291
:106790006091060470910704882777FD8095982FF3
:1067A00026E030E040E050E00E94C4553B014C013F
:1067B00070937308609372086091040470910504EB
:1067C000882777FD8095982F0E94C4555B016C0146
:1067D0007093830860938208E090EB07FF2400E049
:1067E00010E0882477FC8094982CC401B301A801A0
:1067F00097010E94C4553B014C016093450470937E
:1068000046048093470490934804CC24B7FCC0947A
:10681000DC2CC601B5010E94C45560934D047093F1
:106820004E0480934F0490935004609269047092D8
:106830006A0480926B0490926C046093710470936C
:1068400072048093730490937404109275041092F0
:10685000760410927704109278048091140390913A
:106860001503A0911603B0911703909388078093A6
:10687000870710920D0410920C0410927D04109260
:106880007E0410927F041092800480918104909184
:10689000820490938404809383040E94634E82E375
:1068A00090E09093E6038093E5036091040870E024
:1068B00080E090E024EC39E040E050E00E94C455D4
:1068C0006856754C8F4F9F4F609397037093980352
:1068D0008093990390939A036091050870E080E09B
:1068E00090E00E94C4556856754C8F4F9F4F60933F
:1068F0009B0370939C0380939D0390939E0310923F
:10690000B2031092B10360918104709182048827D0
:1069100077FD8095982F2091B3033091B403409177
:10692000B5035091B6030E94C45560937E087093DE
:106930007F08809380089093810810928B041092B6
:106940008A0411E0109301010E94C3518091C00498
:1069500084608093C0048FEF8093E8081092E90868
:1069600080E28093EA08E091DB07F0E0EE0FFF1F82
:10697000EB55F84F8081918182599F4F90938D0400
:1069800080938C04E091DC07F0E0EE0FFF1FEB55E5
:10699000F84F8081918182599F4F90938F0480930B
:1069A0008E04E091DD07F0E0EE0FFF1FEB55F84F8E
:1069B0008081918182599F4F90939104809390049C
:1069C000E091DE07F0E0EE0FFF1FEB55F84F8081FE
:1069D000918182599F4F90939304809392041093D6
:1069E000E80384E680939404DF91CF911F910F9187
:1069F000FF90EF90DF90CF90BF90AF909F908F90DF
:106A00007F906F9008951F93182F11501F3FA9F08A
:106A100080919D04882329F010C080919D048823D3
:106A200061F484E690E09093E6038093E5038AEFB7
:106A300090E00E949A12115080F71F91089588EEFD
:106A40008093DF073EE13093E0078BEF8093E2070E
:106A50008AE08093E3073093E1073093E50793E002
:106A60009093E40758E05093E60720E12093E7076E
:106A700066E06093E8075093E90786EE8093EA07A3
:106A80003093EB0780E88093EC0744E64093ED07F2
:106A900088E78093EE079093EF078EE58093F007E9
:106AA00083E28093F10784E18093F2071092F30769
:106AB0002093F4071092F5071092F6071092F7074B
:106AC0001092F8071092090810920A0810920B0809
:106AD00010920C084093F90788E28093FA0710920D
:106AE000230892E39093FB0786E98093FC0785E0F7
:106AF0008093FD079093FE072AE52093FF0790936C
:106B00000008109222082093010883E48093020871
:106B100086E48093030885E5809304088093050844
:106B200080E28093060880930708909308088FE519
:106B300080930D0883EF80930F0830930E083093F5
:106B400010088DEF809311084093120820931308CA
:106B500020931408209315088BE4809316088093E3
:106B60001708809318081092190860931A08509318
:106B70001B0820931C0830931D0840931E08409367
:106B80001F0884E080932008A8E2B8E0EAE7F3E079
:106B90008CE001900D928150E1F7089588E6809392
:106BA000DF075EE15093E0078BEF8093E2078AE016
:106BB0008093E3075093E1075093E50793E09093A8
:106BC000E4078CE08093E60780E18093E70776E0B6
:106BD0007093E80768E06093E90786EE8093EA0720
:106BE0005093EB0780E88093EC0780E58093ED07F6
:106BF00088E78093EE079093EF078EE58093F00788
:106C000083E28093F1075093F2071092F30730E28A
:106C10003093F4071092F5071092F6071092F707D9
:106C20001092F8071092090810920A0810920B08A7
:106C300010920C0844E64093F90788E28093FA0723
:106C40001092230892E39093FB0786E98093FC0758
:106C500085E08093FD079093FE072AE52093FF07C8
:106C600090930008109222082093010883E48093F7
:106C700002088CE38093030885E5809304088093E1
:106C8000050830930608309307089BE490930808A2
:106C90008FE580930D0883EF80930F0884E1809344
:106CA0000E08809310088DEF80931108409312080E
:106CB0002093130820931408209315089093160826
:106CC00090931708909318081092190870931A0857
:106CD00060931B0820931C0850931D0840931E08C6
:106CE00040931F0884E080932008A8E2B8E0E4E81D
:106CF000F3E08CE001900D928150E1F7089588E671
:106D00008093DF073EE13093E0078BEF8093E2074B
:106D10008AE08093E3073093E1073093E507E4E0EE
:106D2000E093E4075FE05093E6073093E7078CE0D9
:106D30008093E80778E07093E90786EE8093EA078E
:106D40003093EB0780E88093EC0780E58093ED07B4
:106D500026E92093EE0783E08093EF078EE580938A
:106D6000F00783E28093F1073093F2071092F30764
:106D700060E26093F4071092F5071092F607109204
:106D8000F7071092F8071092090810920A0810925B
:106D90000B0810920C0844E64093F90788E28093B0
:106DA000FA071092230892E39093FB072093FC07C5
:106DB00085E08093FD079093FE072AE52093FF0767
:106DC00090930008109222082093010883E4809396
:106DD00002081092030885E5809304088093050853
:106DE00080E18093060860930708409308088FE5C8
:106DF00080930D0883EF80930F0850930E085093F3
:106E000010088DEF80931108409312082093130807
:106E100020931408209315088BE480931608809320
:106E20001708809318081092190886E080931A08B2
:106E300070931B0820931C0830931D0840931E0874
:106E400040931F08E0932008A8E2B8E0ECE8F3E0E4
:106E50008CE001900D928150E1F708952F923F92BE
:106E60004F925F926F927F928F929F92AF92BF925A
:106E7000CF92DF92EF92FF920F931F93CF93DF9306
:106E8000CDB7DEB7AE970FB6F894DEBF0FBECDBF5D
:106E90000E94F323409100014C3008F04FC7299A1B
:106EA00020919B0430919C0480914C08682F70E0E5
:106EB000665F7F4F798B688B6217730714F4398B89
:106EC000288B80919404843608F0EFC380910501EB
:106ED000882349F48091090390910A038F5F9F4FA3
:106EE00011F40C943E498091EA049091EB040097D0
:106EF00009F431C701979093EB048093EA044A3078
:106F000009F430C7443109F42DC728988091BE0494
:106F10009091BF04895E934010F40C949745809142
:106F2000F107E82FF0E0F98BE88BF1E0F0938704AC
:106F3000A091D707B0E0AA0FBB1FFD01E554F84FA1
:106F400011821082E091D8072E2F30E0220F331FDC
:106F5000C9018554984FFC0111821082AB55B84F7E
:106F600011961C921E922B55384FD90111961C92E6
:106F70001E92E091DA07F0E0EE0FFF1FEB55F84F9D
:106F800011821082809179038150809379038091DE
:106F900079038F3F09F4D0C4B0918704BFA3BB230A
:106FA00009F0CAC4B091DF072091A704222311F48D
:106FB0000C949A498091FE0790E068897989861738
:106FC000970714F4998B888B71E0709389048B2F49
:106FD00090E09B878A879FA19923B1F010929A0431
:106FE00010929904109296041092950410929804AD
:106FF000109297048AE580937C08A8E7A09368081C
:107000001092A7041092A6042091450430914604E2
:10701000409147045091480429833A834B835C8311
:1070200040915B0850915C0860915D0870915E082A
:1070300048A759A76AA77BA789819A81AB81BC81A0
:10704000480F591F6A1F7B1F40935B0850935C08D1
:1070500060935D0870935E0820914D0430914E045A
:1070600040914F04509150042D833E834F835887A5
:107070002090620830906308409064085090650842
:10708000220E331E441E551E209262083092630861
:1070900040926408509265084091490450914A0416
:1070A00060914B0470914C0449A35AA36BA37CA339
:1070B00080914E0890914F08A0915008B0915108CE
:1070C000840F951FA61FB71F80934E0890934F08FB
:1070D000A0935008B09351086091510470915204EC
:1070E00080915304909154046D8F7E8F8F8F98A35D
:1070F00080913E0890913F08A0914008B0914108CE
:107100002D8D3E8D4F8D58A1820F931FA41FB51F4B
:1071100080933E0890933F08A0934008B0934108A5
:107120003091A6043987332311F40C94CB4210928A
:10713000550410925604109257041092580410925D
:10714000590410925A0410925B0410925C0410923D
:107150005B0810925C0810925D0810925E08109215
:1071600062081092630810926408109265081092E9
:107170004E0810924F081092500810925108109229
:107180003E0810923F0810924008109241088091EA
:10719000650490916604A0916704B091680480939F
:1071A000690490936A04A0936B04B0936C0480917B
:1071B0006D0490916E04A0916F04B091700480935F
:1071C000710490937204A0937304B09374041092AA
:1071D0000F0410920E041092A5041092A4041092B1
:1071E000A3041092A2045091A7045CA780910E04FE
:1071F00090910F048F3F910509F010F40C94B64262
:10720000B985BB2329F4ECA5EE2311F40C94324686
:107210001092A3041092A2041092A5041092A40448
:107220001EA21092890420915B0830915C08409165
:107230005D0850915E0828A739A74AA75BA7209050
:10724000620830906308409064085090650830915F
:1072500068083DA3332341F41092A3041092A204C2
:107260001092A5041092A40448A559A56AA57BA56F
:107270004093C5045093C6046093C7047093C80438
:107280002092C1043092C2044092C3045092C404BC
:1072900010925504109256041092570410925804FC
:1072A0001092590410925A0410925B0410925C04DC
:1072B00010925D0410925E0410925F0410926004BC
:1072C00010925B0810925C0810925D0810925E08A4
:1072D0001092620810926308109264081092650878
:1072E00010924E0810924F081092500810925108B8
:1072F00010923E0810923F081092400810924108E8
:1073000010920F0410920E04E0909904F0909A04E9
:107310006701F7FE02C00C94C54270E1C716D104A4
:1073200064F088EE93E090939603809395038A85AA
:1073300084FD03C081E08093DB040091E807B7017E
:10734000882777FD8095982F202F30E040E050E08F
:107350000E94C4559601442737FD4095542F0E9442
:10736000C45520E032E040E050E00E94385610E082
:107370000E9DB0010F9D700D1E9D700D112477FFA5
:1073800002C00C949B457595679575956795260F7A
:10739000371FA901662757FD6095762F488F598FB3
:1073A0006A8F7B8F4093FC045093FD046093FE042E
:1073B0007093FF048091750490917604A0917704F6
:1073C000B0917804841B950BA60BB70B80937504C2
:1073D00090937604A0937704B0937804813553ECAE
:1073E000950750E0A50750E0B50714F40C94A142AE
:1073F00080E593ECA0E0B0E0809375049093760470
:10740000A0937704B0937804209081043090820494
:107410002114310409F4A8C47A8573FFA5C46981D5
:107420007A818B819C8120E032E040E050E00E9434
:107430003856890137FF02C00C9452496D817E8114
:107440008F81988520E032E040E050E00E9438567D
:10745000690137FF02C00C944C49C016D10614F4E0
:107460000C94E54840907E0850907F08609080081A
:10747000709081088091B3039091B403A091B503FB
:10748000B091B6038C8B9D8BAE8BBF8B80907708B1
:1074900090907808C40197FE02C00C945749813837
:1074A000910514F00C94E848ACE1B2E02A0E3B1EC2
:1074B00071010027F7FC0095102FE4EEFDEF2E0E72
:1074C0003F1EC301B2012C893D894E895F890E940C
:1074D0003856E21AF30A040B150BC801B70128E667
:1074E00031E040E050E00E943856645B70408B0110
:1074F000000F111F000F111F000F111F2091DB043F
:10750000E0909503F0909603E114F10491F4F9E111
:10751000CF16D10474F480918A0490918B04860F65
:10752000971F90938B0480938A04222311F00C946C
:10753000864AB601D7FE02C00C94CE497595679570
:1075400075956795759567956F5F7F4FC8010E9428
:1075500003569B01A901662757FD6095762F440DC0
:10756000551D661D771D40937E0850937F086093DC
:107570008008709381088091A503A82EBB24CA9C23
:107580009001CB9C300DDA9C300D112437FF02C0E6
:107590000C94CA49359527953595279535952795A6
:1075A00035952795359527956501C21AD30AD7FEDB
:1075B00002C00C94C249E114F10411F00C949149F9
:1075C0006090BC047090BD048091BA049091BB049B
:1075D000680E791E77FE02C00C94E54C7594679492
:1075E0007594679475946794A0E4B0E06A0E7B1E6E
:1075F0008091830490918404AA2797FDA095BA2FC7
:10760000ECE1EE2EE2E0FE2E012D112DE81AF90A32
:107610000A0B1B0BCB01BA012C893D894E895F896E
:107620000E943856E20EF31E041F151FC801B70151
:1076300028E631E040E050E00E943856645B70403C
:107640006C9DC0016D9D900D7C9D900D1124B3012A
:107650000E9403569501220F331F2A0D3B1D26174A
:10766000370714F40C94D249309521953F4F621797
:1076700073070CF4B9019B01442737FD4095542F43
:107680008091750490917604A0917704B09178046C
:10769000820F931FA41FB51F8093750490937604E7
:1076A000A0937704B093780463C3809194048D38D9
:1076B00008F468CC109287048091F20722E3829F3D
:1076C000C00111249093EB048093EA04E889F989BE
:1076D000B9978CF080919D04882369F08091BE0455
:1076E0009091BF04FFEF8F3F9F0779F00196909331
:1076F000BF048093BE048091BE049091BF048F3F6D
:10770000910509F010F40C9407498091C00482603F
:107710008093C0048091D907A82FB0E0AA0FBB1FA7
:10772000FD01EB55F84F80819181813591050CF475
:10773000C4C080919D04882309F0BFC08091DA07FE
:10774000E82FF0E0EE0FFF1FEB55F84F808191819D
:107750008C34910514F40C94EC498091E9048F5F0A
:107760008093E904893C08F4A8C04C3010F00C94D4
:10777000174E299810929D041092E9041092BF04AC
:107780001092BE048091D707282F30E0220F331FBC
:10779000F901EB55F84F808191818734910514F4FC
:1077A0000C94024E8091D807A82FB0E0AA0FBB1FFF
:1077B000AD014B55584FFA01808191818734910575
:1077C0002CF0F901EB55F84F80819181FA0180810D
:1077D00091818734910514F40C94EC4DF901EB552B
:1077E000F84F808191818734910514F40C94EC4D0D
:1077F00042E0FD01EB55F84F80819181863491057F
:107800004CF4F901EB55F84F808191818734910553
:107810000CF043E0FD01EB55F84F808191818A5BCC
:107820009F4F4CF4F901EB55F84F808191818734DB
:1078300091050CF044E0AB55B84F8D919C918A5B5B
:107840009F4F4CF42B55384FD9018D919C91863424
:1078500091050CF445E0842F0E94B0028091D80776
:10786000A82FB0E0AA0FBB1FAB55B84F8D919C91CC
:1078700097FF02C00C94244E4E9714F00C94B74D11
:10788000E091D707F0E0EE0FFF1FEB55F84F808136
:1078900091818A5B9F4F14F00C94B74D81E08093E7
:1078A0009A0688EE93E09093E6038093E503809137
:1078B000D907A82FB0E0AA0FBB1FAB55B84F8D91C9
:1078C0009C918B5A9F4F0CF05DCB8091DA07C82EAC
:1078D000DD24CC0CDD1CF601EB55F84F8081918145
:1078E000855B9F4F14F00C94A6498091E8048F5F4C
:1078F0008093E804893C10F00C94AB4A65EA77E089
:10790000C60ED71ED6018D919C918C34910514F42E
:107910000C94AA498091E7048F5F8093E704893C27
:1079200008F430CB10929D0488EC8093E704109209
:10793000BF041092BE0426CB0E947E2C8091D707F4
:10794000A82EBB24AA0CBB1CF501EB55F84F2081D7
:1079500031818091E607882E9924F501E554F84F8E
:107960000190F081E02D8091E707682F70E0289D5D
:10797000A001299D500D389D500D11242091D10456
:107980003091D204C901880F991F820F931F480FAD
:10799000591F57FF02C00C94FF489A01359527954F
:1079A00035952795E69FC001E79F900DF69F900DB6
:1079B0001124280F391F3093D2042093D1048091D1
:1079C00024059091250540912005509121056901DC
:1079D000C81AD90AC41AD50AD0929604C09295043E
:1079E0008091D807E82EFF24EE0CFF1CF701EB5521
:1079F000F84F80819181F701E554F84F0190F081B3
:107A0000E02D889DA001899D500D989D500D112459
:107A10002091CF043091D004C901880F991F820FA3
:107A2000931F480F591F57FF02C00C9403499A0136
:107A30003595279535952795E69FC001E79F900DD1
:107A4000F69F900D1124280F391F3093D0042093F6
:107A5000CF048091260590912705409122055091F1
:107A600023058901081B190B041B150B109398049F
:107A700000939704E091DA07F0E0EE0FFF1FEB555B
:107A8000F84F80819181909581959F4F90939A04B2
:107A900080939904833091050CF452C1029790931E
:107AA0009A0480939904E091D907F0E0EE0FFF1F4C
:107AB000EB55F84F6080718028E730E0620E731E4E
:107AC00070929C0460929B046091A70370E08827E9
:107AD00077FD8095982F0E940C5520E030E040E221
:107AE00051E40E9475540E94DE5460937C083091EA
:107AF000A803309368088091A60680FF06C0809195
:107B00008608813810F00C94D54580919B049091A3
:107B10009C0497FF02C00C947549B091DF07B2FF37
:107B200002C010926808209195043091960440910B
:107B3000BA045091BB04C90137FF02C00C948049BC
:107B4000959587959595879597FF02C00C947B49ED
:107B5000481759070CF02AC7C90137FF02C00C9417
:107B6000BD4997FF02C00C94BA49959587959595A4
:107B700087959093BB048093BA048536910514F0E1
:107B80000C94CD4520919704309198044091BC0409
:107B90005091BD04C90137FF02C00C9483499595EB
:107BA00087959595879597FF02C00C948C49481747
:107BB00059070CF0F4C6C90137FF02C00C94B5494F
:107BC00097FF02C00C94B249959587959595879536
:107BD0009093BD048093BC04853691050CF0D6C704
:107BE000E0918704EFA3EE2341F01092BB041092C2
:107BF000BA041092BD041092BC04F701EB55F84F83
:107C0000208131818091FF07482F50E042175307B0
:107C100024F48091220882FDB5C7F701EB55F84F97
:107C20002081318180910008BA01681B71092617F3
:107C3000370714F41092A804F701EB55F84F808130
:107C4000918166277727641B750B8617970724F4A5
:107C50008091220883FD92C78091A904882389F02E
:107C600085EA97E0E80EF91EF701208131818091C5
:107C7000000890E0841B950B8217930714F40C9472
:107C80003A49F501EB55F84F808191814817590722
:107C900024F48091220880FD6DC7A091AB04AA2333
:107CA00079F0F501EB55F84F208131818091000882
:107CB000FA01E81BF1092E173F0714F40C9431491F
:107CC000F501EB55F84F808191818617970724F4D1
:107CD0008091220881FD4AC78091AA04882389F0F7
:107CE00025EA37E0A20EB31EF50120813181809193
:107CF000000890E0841B950B8217930714F40C94F2
:107D000036498091A804882329F48091A904882306
:107D100009F429C7F1E0F093A704AA2329F480917C
:107D2000AA04882309F41BC781E08093A60410925B
:107D3000A7041092A8041092A9043CC92998B0C8BD
:107D4000EFEF8E3F9E070CF087C7029690939A0440
:107D500080939904A8CE10929D04109287044A3013
:107D600009F0D0C8289AD2C88090770890907808F7
:107D70008091DC0481508093DC048F3F09F45DC561
:107D8000BEA1BB2381F01092000510920105109254
:107D90000205109203051092040510920505109239
:107DA000060510920705E985EE2309F4B5C31F8681
:107DB0001E86442455242CA5222309F498C31D862D
:107DC0001C86222433248091390890913A08893CFA
:107DD00091050CF480C388EC90E090933A0880936E
:107DE000390860914308709144087EA76DA7693CEB
:107DF00071050CF461C3A8ECB0E0BEA7ADA7B093C9
:107E00004408A0934308A0907C08BB24CC24DD2424
:107E10007C010027F7FC0095102FEE0CFF1C001FC3
:107E2000111FEE0CFF1C001F111FEE0CFF1C001F8A
:107E3000111FEE0CFF1C001F111FEE0CFF1C001F7A
:107E4000111FEE0CFF1C001F111FEE0CFF1C001F6A
:107E5000111F60904608709047089301442737FD32
:107E60004095542FC601B5010E94C455E60EF71E79
:107E7000081F191FC801B70120E430E040E050E0BE
:107E80000E9438563201620E731E7092470860924B
:107E900046086DA57EA57B010027F7FC0095102FF5
:107EA000EE0CFF1C001F111FEE0CFF1C001F111F0A
:107EB000EE0CFF1C001F111FEE0CFF1C001F111FFA
:107EC000EE0CFF1C001F111FEE0CFF1C001F111FEA
:107ED000EE0CFF1C001F111F409036085090370811
:107EE000B201882777FD8095982FA60195010E9401
:107EF000C455E60EF71E081F191FC801B70120E47C
:107F000030E040E050E00E9438562101420E531EFE
:107F10005092370840923608880C991CB401882783
:107F200077FD8095982FA60195010E94C45520E405
:107F300030E040E050E00E94385679018A01ADA15E
:107F40006A2F70E080E090E020916104309162043B
:107F500040916304509164040E94C45520EF35E5BC
:107F600040E050E00E9438564701820E931E9092E6
:107F7000780880927708B1E06B16B0E47B060CF4C9
:107F80008DC2612C40E4742E7092470860924608BE
:107F9000F1E04F16F0E45F060CF472C2412C20E4CD
:107FA000522E509237084092360831E0831630E462
:107FB00093060CF457C2812C80E4982E9092780896
:107FC0008092770868897989660F771F660F771F17
:107FD0007EA76DA77A8570FF2CC071FFEEC48091DB
:107FE000220884FD02C00C94EE488091A2038155C2
:107FF0008B3310F00C94F4488091B7038150809338
:10800000B7038F3F11F40C94DB4B20919E04309109
:108010009F04F2C4EDA5FEA5E217F30724F4F09344
:10802000E604E093E5042091E5043091E6043EA7E0
:108030002DA780917608282E3324A101440F551FC7
:10804000440F551FCA01805590400DA51EA58017ED
:1080500091070CF48C011093500700934F07688D23
:10806000798D8A8D9B8D660F771F881F991F660FEC
:10807000771F881F991F7401E61AF70A013A110544
:108080000CF4E2C19801359527952E153F0584F033
:10809000F80117FF02C00C945D49F595E79522277A
:1080A00033272E1B3F0B2E153F0514F40C94E2488A
:1080B000CA01801B910B821793070CF49C01C80125
:1080C000841B950B5901281739070CF45C0180912A
:1080D0009504909196046301C81AD90AD0925A085F
:1080E000C0925908ADA1AA2309F494C1EE85FF8579
:1080F000E81BF90BCF01AA2797FDA095BA2F209175
:108100000405309105054091060550910705280F9B
:10811000391F4A1F5B1F20930405309305054093C8
:108120000605509307052130FAEF3F07F0E04F07AF
:10813000F0E05F070CF458C120E03AEF40E050E077
:1081400020930405309305054093060550930705D9
:1081500080919F039091A0033C01882477FC809438
:10816000982CCA01B901A40193010E943856C20E8D
:10817000D31EB501B7FCE6C477FDE1C475956795DC
:10818000600F711F882777FD8095982F2091B0038D
:1081900030E040E050E00E94C45520E430E040E090
:1081A00050E00E9438567901C216D3060CF49601AD
:1081B000CC24DD24CE18DF08DB8ACA8AC216D30697
:1081C0000CF469018091970490919804481A590A17
:1081D00050923508409234087DA1772309F4EAC013
:1081E000AC85BD85A81BB90BFD01CF01AA2797FD62
:1081F000A095BA2F2091000530910105409102050C
:1082000050910305280F391F4A1F5B1F209300055B
:108210003093010540930205509303052130FAEF96
:108220003F07F0E04F07F0E05F070CF4ADC020E03F
:108230003AEF40E050E02093000530930105409371
:10824000020550930305CA01B901A40193010E94DC
:108250003856B201620F731F97016E157F050CF43B
:108260009B0179018A899B89281739070CF47C01C5
:108270004501800E911E6091E3047091E404C601F3
:10828000880D991D0E94DD239093E4048093E304FC
:1082900097FD5FC49C01359527953595279580916D
:1082A0004C08682E7724261537050CF066C0C301EC
:1082B000809338086091E1047091E204C4018C1944
:1082C0009D090E94DD239093E2048093E10497FDD1
:1082D0003EC49595879595958795861597050CF0DD
:1082E00046C0C301809345086091DF047091E004AB
:1082F000C8018A199B098E0D9F1D0E94DD23909352
:10830000E0048093DF0497FD28C4959587959595A3
:1083100087958615970534F5C30180936E086091A3
:10832000DD047091DE040E191F09C8018A199B092A
:108330000E94DD239093DE048093DD0497FD0BC43F
:1083400095958795959587958615970514F40C94C2
:10835000484E3C012816390614F00C94484E310161
:108360000C94484E28163906C4F6C101D6CF2816FB
:1083700039060CF0B7CFC101B5CFC90122163306BB
:108380000CF096CFC10194CF203066E036076FEF36
:1083900046076FEF56070CF056CF20E036E04FEF60
:1083A0005FEF209300053093010540930205509341
:1083B000030549CFC201AA2797FDA095BA2F2091A6
:1083C0000005309101054091020550910305280FE9
:1083D000391F4A1F5B1F209300053093010540930E
:1083E0000205509303051ACF203066E036076FEF81
:1083F00046076FEF56070CF0ABCE20E036E04FEFAC
:108400005FEF2093040530930505409306055093D4
:1084100007059ECEC601AA2797FDA095BA2F2091E9
:108420000405309105054091060550910705280F78
:10843000391F4A1F5B1F20930405309305054093A5
:108440000605509307056FCE97017FEF203B370756
:1084500014F420EB3FEF213531050CF429CE20E553
:1084600030E026CE40E0841640EC94060CF0AACD15
:10847000812C00EC902E9092780880927708A2CD03
:1084800020E0421620EC52060CF08FCD412C90ECEF
:10849000592E509237084092360887CDE0E06E168C
:1084A000E0EC7E060CF074CD612C30EC732E7092F3
:1084B0004708609246086CCDEDA5FEA5E853FF4F36
:1084C0000CF0A1CC48E35FEF5EA74DA750934408A2
:1084D0004093430898CC4FEF883394070CF081CC3D
:1084E00088E39FEF90933A08809339087ACC3DA1B6
:1084F000632F70E080E090E02D813E814F815885B0
:108500000E94C45528EF3AE240E050E00E943856FD
:108510003D872C87190157CCFDA16F2F70E080E0BB
:1085200090E029813A814B815C810E94C45528EFFB
:108530003AE240E050E00E9438563F872E872901FA
:108540003ACC805B9C43AF4FBF4F14F00C94043A7D
:1085500080EB9CE3AFEFBFEF8093750490937604BC
:10856000A0937704B09378040C94043A5091890452
:108570005EA3609168086DA3E0909904F0909A045E
:108580006701F7FC02C00C948D39CC24DD24CE1891
:10859000DF080C948D394091A7044CA7442309F4BB
:1085A0005EC0109255041092560410925704109217
:1085B00058041092590410925A0410925B041092BD
:1085C0005C0410925B0810925C0810925D08109297
:1085D0005E0810926208109263081092640810926C
:1085E000650810924E0810924F0810925008109291
:1085F000510810923E0810923F08109240081092C5
:1086000041088091650490916604A0916704B0913F
:1086100068048093690490936A04A0936B04B093F8
:108620006C0480916D0490916E04A0916F04B091E0
:1086300070048093710490937204A0937304B093B8
:10864000740410920F0410920E041092A50410925C
:10865000A4041092A3041092A2040C94F638809102
:108660008507909186078150924014F40C94F63857
:108670008091E8088F3F11F40C94394BE090EB07A0
:10868000FF2400E010E0A82EBB24A7FCB094CB2C64
:10869000DB2C69817A818B819C81A80197010E94E2
:1086A00038568091720890917308AA2797FDA0957B
:1086B000BA2F281B390B4A0B5B0BCA01B901A60163
:1086C00095010E94C45520E032E040E050E00E9455
:1086D000385639014A016D817E818F819885A801C4
:1086E00097010E9438568091820890918308AA27AA
:1086F00097FDA095BA2F281B390B4A0B5B0BCA01BB
:10870000B901A60195010E94C45520E032E040E085
:1087100050E00E94385659016A018091BA04909144
:10872000BB04813491050CF0CBC58091BC049091C1
:10873000BD04813491050CF0C3C5E091DA07F0E087
:10874000EE0FFF1FEB55F84F0190F081E02DF7FF82
:1087500002C00C94B84C7A97A4F0C401B30123E092
:1087600030E040E050E00E94385639014A01C6012D
:10877000B50123E030E040E050E00E943856590156
:108780006A018091EA08E82EFF24E7FCF0940F2D9F
:108790001F2DA4019301E614F7040805190514F42C
:1087A000A8019701992787FD9095909581959F4FF6
:1087B000AA2797FDA095BA2F39014A012817390732
:1087C0004A075B0714F43C014D01EA14FB040C0555
:1087D0001D0514F457016801A816B906CA06DB0680
:1087E00014F45C016D018091650490916604A09180
:1087F0006704B091680486199709A809B90980939C
:10880000650490936604A0936704B0936804809114
:108810006D0490916E04A0916F04B09170048A1958
:108820009B09AC09BD0980936D0490936E04A093DD
:108830006F04B09370040C94F63888E18093DC04E4
:10884000E090EB07FF24EE0CFF1CEE0CFF1C002752
:10885000F7FC0095102F69817A818B819C81A8019A
:1088600097010E94385630934207209341076D814B
:108870007E818F819885A80197010E943856309398
:10888000440720934307809172089091730897FDE5
:1088900067C595958795959587959093460780939D
:1088A0004507809182089091830897FD57C595955B
:1088B0008795959587959093480780934707909261
:1088C0004A078092490720919E0430919F0430937B
:1088D0004C0720934B0760917D0470917E0480913A
:1088E0007F049091800420E032E040E050E00E945C
:1088F000385630934E0720934D07309252072092FE
:10890000510780910E0390910F0390935407809329
:10891000530760917E0870917F0880918008909144
:1089200081082091B3033091B4034091B503509175
:10893000B6030E943856309358072093570780910A
:10894000940490E0909356078093550780919A067F
:1089500090E090936807809367078091E903909176
:10896000EA0390936A07809369078091E908992741
:1089700087FD9095909378078093770780912005E5
:108980009091210590937E0780937D078091220529
:10899000909123059093800780937F07F1C9415000
:1089A00050405093BD044093BC041AC941505040FC
:1089B0005093BB044093BA04E5C88091A203209170
:1089C000B1033091B203280F311D8091E40790E08C
:1089D000FC012E9FC0012F9F900D3E9F900D1124F2
:1089E00044979093A1048093A00481E0809388042D
:1089F00020919E0430919F04FFA1FF2321F010924B
:108A0000A1041092A0044091A0045091A104421727
:108A100053070CF00ECB80918804882309F409CB0E
:108A20008091A30390E0241B350BAC01429FC00151
:108A3000439F900D529F900D112497FDDBC65C0162
:108A4000B594A794B594A794C0900C04D0900D044D
:108A500060917D0470917E0480917F0490918004E8
:108A6000E090A403FF2400E010E020E830E040E0C4
:108A700050E00E943856C801B7010E94C45520E258
:108A800030E040E050E00E943856A901285E3E4F99
:108A900014F448EE5EEF2091E5043091E604C9013C
:108AA000880F991F820F931FBC01660F771F660FF7
:108AB000771F680F791F9601D7FCA1C635952795BA
:108AC000CB01821B930B9A014951514014F028E1CC
:108AD00031E0821B930B9C018DA59EA58A199B09F1
:108AE000280F391F37FD88C6359527953595279569
:108AF00035952795359527953093E6042093E50421
:108B00008091E007682F70E0660F771F660F771F70
:108B1000261737070CF07ECA8DA59EA586179707E6
:108B20000CF49FC57093E6046093E5047CCA109230
:108B30009D040C94C2376D5F7F4F0C94C3396F5FF7
:108B40007F4F1CCB662777276A197B0915CB0396C5
:108B5000C0CB03969FCB0396F3CB0396D6CB109254
:108B6000A6040C94D4371092A704D7C881E0809350
:108B7000AA04C7C8A1E0A093AB04A2C881E0809377
:108B8000A9047FC881E08093A80456C884E690E0D9
:108B90009093BD048093BC0423C884E690E0909336
:108BA000BB048093BA040C94C23D80919F06992720
:108BB00087FD9095AC01489DC001499D900D589D41
:108BC000900D1124C80ED91ED0929604C09295041F
:108BD0008091A006992787FD9095BC01689DC001F2
:108BE000699D900D789D900D1124080F191F109309
:108BF0009804009397042091A106332727FD309510
:108C00008091990490919A04820F931F90939A04F3
:108C1000809399042091E40730E08091A30699277E
:108C200087FD9095DC012A9FC0012B9F900D3A9FF4
:108C3000900D11249093B2038093B1038091A2060A
:108C400090E08615970514F00C94853D90939C0454
:108C500080939B040C94853D10929A041092990481
:108C60000C94533DF0918904FEA3FF2311F00C9462
:108C70000839209107082C8F222311F40C9408390D
:108C800040915B0850915C0860915D0870915E08AE
:108C9000CB01BA0120E031E040E050E00E943856BC
:108CA00028A739A74AA75BA720935B0830935C08E5
:108CB00040935D0850935E082090620830906308EE
:108CC0004090640850906508C201B10120E031E095
:108CD00040E050E00E94385619012A0120936208B2
:108CE000309363084093640850936508E090EB0765
:108CF000FF2400E010E0209155043091560440918B
:108D0000570450915804C801B7010E94C45520E08F
:108D100031E040E050E00E94385659016A0120934A
:108D200055043093560440935704509358042091AF
:108D3000590430915A0440915B0450915C04C8017D
:108D4000B7010E94C45520E031E040E050E00E94AD
:108D5000385639014A012093590430935A044093FC
:108D60005B0450935C0460915D0470915E0480919B
:108D70005F049091600420E031E040E050E00E9408
:108D8000385620935D0430935E0440935F04509303
:108D90006004E0900608FF2400E010E068A579A5D3
:108DA0008AA59BA56A197B098C099D09A8019701D1
:108DB0000E9438562093D7043093D8044093D904A6
:108DC0005093DA04CA01B90120E031E040E050E0FC
:108DD0000E94385669013093A5042093A404C2016F
:108DE000B1016619770988099909A80197010E94BC
:108DF0003856CA01B90120E031E040E050E00E945D
:108E00003856B9013093A3042093A2048091BA0488
:108E10009091BB0481349105ACF48091BC04909195
:108E2000BD048134910574F4E091DA07F0E0EE0FAF
:108E3000FF1FEB55F84F0190F081E02DF7FD17C7AC
:108E40007A972CF08091E8088F3F09F4C8C66091AA
:108E50004E0870914F08809150089091510820E081
:108E600031E040E050E00E94385620934E083093A5
:108E70004F08409350085093510860913E087091FC
:108E80003F08809140089091410820E031E040E0A7
:108E900050E00E94385620933E0830933F0840939C
:108EA000400850934108E9A0FAA00BA11CA16981D8
:108EB0007A818B819C81E61AF70A080B190BE092E4
:108EC000F804F092F9040093FA041093FB04AD8CBB
:108ED000BE8CCF8CD8A08D819E81AF81B885A81A19
:108EE000B90ACA0ADB0AA092F404B092F504C0924F
:108EF000F604D092F704E092F004F092F1040093AB
:108F0000F2041093F304A092EC04B092ED04C0922A
:108F1000EE04D092EF048091690490916A04A091CC
:108F20006B04B0916C048E199F09A00BB10B809358
:108F3000690490936A04A0936B04B0936C048091CD
:108F4000710490917204A0917304B09174048A1911
:108F50009B09AC09BD098093710490937204A0939E
:108F60007304B093740420918A0430918B042138E7
:108F7000310594F0809133049091340401969093DC
:108F800034048093330480916608909167080196B9
:108F9000909367088093660820583F4F94F480911F
:108FA00033049091340401979093340480933304F4
:108FB0008091660890916708019790936708809365
:108FC000660810928B0410928A0481E090E09093DE
:108FD000CE048093CD048091C5049091C604A091E5
:108FE000C704B091C80428A539A54AA55BA5821B72
:108FF000930BA40BB50B815E914BAF4FBF4F8F53BB
:109000009C49A040B04008F457C49090E90848E15A
:1090100049150CF453C41092CE041092CD0488EE7E
:1090200093E090939603809395039C8D692E77240B
:109030008091CD049091CE046816790624F4709244
:10904000CE046092CD04992079F0292D332727FD95
:1090500030958091CD049091CE042817390724F4DF
:109060003093CE042093CD04A1E0EA16A4E0FA06E2
:10907000A0E00A07A0E01A0774F080912F049091F5
:1090800030042091CD043091CE04820F931F909331
:10909000300480932F04B0E0EB16BCEFFB06BFEF6B
:1090A0000B07BFEF1B0774F480912F0490913004DD
:1090B0002091CD043091CE04821B930B9093300409
:1090C00080932F0481E090E09093CE048093CD04B0
:1090D0001092D3041092D4041092D5041092D604A6
:1090E0008091C1049091C204A091C304B091C404C2
:1090F00082199309A409B509815E914BAF4FBF4F07
:109100008F539C49A040B04008F47CC3F8E1F915A6
:109110000CF478C31092CE041092CD0488EE93E044
:1091200090939603809395038091CD049091CE0403
:109130006816790624F47092CE046092CD049920CA
:1091400079F0292D332727FD30958091CD0490911A
:10915000CE042817390724F43093CE042093CD048D
:1091600071E0A71674E0B70670E0C70670E0D70696
:1091700074F080913104909132042091CD043091AB
:10918000CE04820F931F909332048093310480E0C9
:10919000A8168CEFB8068FEFC8068FEFD80614F02C
:1091A0000C94273980913104909132042091CD04A0
:1091B0003091CE04821B930B909332048093310440
:1091C0000C94273997010C94584068010C94323A5A
:1091D00060E070E000E010E00C947E3A8091A20321
:1091E000823310F40C94FC3F81E08093880488EC77
:1091F0008093B70320919E0430919F04FDCB4D5F77
:109200005F4F0C94CD3C4D5F5F4F0C94173D109217
:10921000040510920505109206051092070510929C
:1092200000051092010510920205109203058A3F75
:10923000910511F00C948A3B81E08093DB0410923D
:10924000FC041092FD041092FE041092FF04109290
:1092500075041092760410927704109278040C949E
:109260008A3BA0E01092AB040C94603E1092AA04DA
:109270000C94813E1092A9040C94413E88E99AE333
:109280009093E6038093E50380E09CE090930A03CB
:10929000809309030C947337D094C194D108D3946C
:1092A0000C942D3A109501951F4F0C941E3A882767
:1092B0009927881999090C944F3A31960C944D408E
:1092C000C401B30122E030E040E050E00E94385693
:1092D00039014A01C601B50122E030E040E050E02A
:1092E0000E94385659016A0128CA10929C041092B3
:1092F0009B040C948D3D909581959F4F0C94A83DB7
:1093000003960C94A03D0396959587959595879522
:1093100097FD02C00C94D73D909581959F4F0C947A
:10932000D73D0894E108F108F0929603E092950386
:109330000C94B83E4B2F50E05B874A878091A6047F
:10934000882311F40C94EB370C94DA371092E8046C
:109350000C947E3C1092E7040C94C2370396A7CA83
:10936000039697CA03960C94E43D909581959F4F80
:109370000C94E03D03960C94B53D909581959F4FDC
:109380000C94B13D84EF91E0909396038093950304
:109390000C94B83E215E3F4F0C94CA3A695F7F4FF0
:1093A0000C949E3A442737FD4095542F80917504C4
:1093B00090917604A0917704B0917804820F931F66
:1093C000A41FB51F8093750490937604A09377042F
:1093D000B09378040C94B83E80819181855B9F4F57
:1093E0000CF005C38091E9048F5F8093E904893C08
:1093F00010F40C945D3C4C3008F024C429988FEF95
:1094000004E010E0D801082E0E945B5610929D04E3
:109410001092E9041092BF041092BE040E9486329A
:109420008091390490913A0497FD28C4892F990FAF
:10943000990BD801082E0E945B56809139049091B7
:109440003A0460E071E00E9403560F5F1F4FD8019D
:10945000082E0E945B560150104020913B04309131
:109460003C0437FD08C4832F992787FD9A950E5F2A
:109470001F4FD801082E0E945B5680913B049091AB
:109480003C0460E071E00E9403560F5F1F4FD8015B
:10949000082E0E945B560350104060913F0470916B
:1094A000400480914104909142040E94D9549B0150
:1094B00077FDE7C3832F992787FD9A950C5F1F4F90
:1094C000D801082E0E945B5660913F0470914004C1
:1094D00080914104909142040E94D954DC01CB0157
:1094E00060E071E00E9403560F5F1F4FD801082E05
:1094F0000E945B560E94BC020E9403358091D907EE
:10950000A82FB0E0AA0FBB1F0C945D3C88EC90E044
:109510009093E6038093E503B101882777FD80955A
:10952000982F2C893D894E895F890E94C4552B0153
:109530003C0160937E0870937F088093800890932D
:1095400081080E943856309384042093830410923B
:10955000DB040C94993A88EC8093E80481E090E075
:109560009093BF048093BE0481E080939D04109289
:10957000FC041092FD041092FE041092FF0410925D
:109580007504109276041092770410927804109269
:10959000790410927A0410927B0410927C04E0907B
:1095A000EB07FF2400E010E06091720870917308EF
:1095B000882777FD8095982FA80197010E94C455B0
:1095C00060936504709366048093670490936804C5
:1095D0006091820870918308882777FD8095982F85
:1095E0000E94C45560936D0470936E0480936F0461
:1095F000909370048091450490914604A091470493
:10960000B09148048093690490936A04A0936B041A
:10961000B0936C0480914D0490914E04A0914F043E
:10962000B09150048093710490937204A0937304DA
:10963000B09374041092040510920505109206056B
:109640001092070510920005109201051092020574
:10965000109203058091C00488608093C0040C942C
:109660007E3CADA5BEA5B093E604A093E5040C94A2
:109670001340E090EB07FF2400E010E069817A815D
:109680008B819C81A80197010E94385659016A017B
:109690008091720890917308AA2797FDA095BA2F20
:1096A000A81AB90ACA0ADB0A6D817E818F81988562
:1096B000A80197010E94385679018A018091820899
:1096C00090918308AA2797FDA095BA2FE81AF90A66
:1096D0000A0B1B0BC601B50120E130E040E050E071
:1096E0000E94385639014A01C801B70120E130E033
:1096F00040E050E00E94385659016A018091BA0456
:109700009091BB04813491053CF48091BC0490910C
:10971000BD0481349105A4F0C401B30123E030E01D
:1097200040E050E00E94385639014A01C601B501B7
:1097300023E030E040E050E00E94385659016A01D1
:10974000E091DA07F0E0EE0FFF1FEB55F84F0190C4
:10975000F081E02DF7FD29C27A97A4F0C401B3018E
:1097600023E030E040E050E00E94385639014A01E1
:10977000C601B50123E030E040E050E00E943856D9
:1097800059016A0171E267167104810491040CF4B5
:1097900009C180E2682E712C812C912C91E2A916CE
:1097A000B104C104D1040CF4E8C010E2A12EB12C24
:1097B000C12CD12C18C88091180390911903895E8F
:1097C000934008F408C190910B049A5090930B04B5
:1097D00080919007891B87BD8CE291E09093E6030E
:1097E0008093E5038AEF8093B70320919E04309124
:1097F0009F0402C9039623C9215F3F4F75C92F5F9C
:109800003F4F5CC921E0A21620E1B20620E0C2066B
:1098100020E0D2060CF44DC18091CA04882309F4DB
:109820000DC2D601C50149E0B595A79597958795D5
:109830004A95D1F701969093CE048093CD04D6013A
:10984000C50133E0B595A795979587953A95D1F7DA
:109850008093D3049093D404A093D504B093D604FA
:1098600089589341A040B04064F088E893E1A0E0BB
:10987000B0E08093D3049093D404A093D504B09324
:10988000D6046091D3047091D4048091D504909152
:10989000D60420E031E040E050E00E94385680914C
:1098A000A2049091A304820F931F9093A30480932A
:1098B000A2041092C90438CC9090E90851E0E51652
:1098C00050E1F50650E0050750E015070CF493C091
:1098D0008091CC04882309F4ADC1D801C70179E097
:1098E000B595A795979587957A95D1F70196909319
:1098F000CE048093CD04D801C70163E0B595A79548
:10990000979587956A95D1F78093D7049093D8045B
:10991000A093D904B093DA0489589341A040B04091
:1099200064F088E893E1A0E0B0E08093D7049093DE
:10993000D804A093D904B093DA046091D70470914D
:10994000D8048091D9049091DA0420E031E040E01D
:1099500050E00E9438568091A4049091A504820F93
:10996000931F9093A5048093A4041092CB045DCB25
:10997000F095E195FF4F0C94AB43A0EEAA16AFEF24
:10998000BA06AFEFCA06AFEFDA0614F00C94F34351
:10999000B0EEAB2EBFEFBB2EBFEFCB2EBFEFDB2E5B
:1099A0000C94F34380EE68168FEF78068FEF8806ED
:1099B0008FEF98060CF0F2CE00EE602E0FEF702EB7
:1099C0000FEF802E0FEF902EE9CE87E090E0680E2B
:1099D000791E0C94EE3A8091180390911903843605
:1099E000910508F0E6C090910B04965FEFCE1092BF
:1099F000E9040C945D3C1092CC0470E0E71670EF23
:109A0000F7067FEF07077FEF17070CF0AECF8091C7
:109A1000CB04882309F421C188279927DC018E19FA
:109A20009F09A00BB10B59E0B595A7959795879520
:109A30005A95D1F701969093CE048093CD04C80136
:109A4000B70128E030E040E050E00E943856209313
:109A5000D7043093D8044093D9045093DA0428579C
:109A60003C4E4F4F5F4F64F488E79CEEAFEFBFEF83
:109A70008093D7049093D804A093D904B093DA04C8
:109A80006091D7047091D8048091D9049091DA0440
:109A900020E031E040E050E00E9438568091A4047C
:109AA0009091A504820F931F9093A5048093A40422
:109AB000BCCA1092CA0440E0A41640EFB4064FEFAF
:109AC000C4064FEFD4060CF0F4CE8091C90488236D
:109AD00009F4BFC088279927DC018A199B09AC09C2
:109AE000BD0929E0B595A795979587952A95D1F752
:109AF00001969093CE048093CD04C601B50128E071
:109B000030E040E050E00E9438562093D304309378
:109B1000D4044093D5045093D60428573C4E4F4F5D
:109B20005F4F64F488E79CEEAFEFBFEF8093D30400
:109B30009093D404A093D504B093D6046091D30439
:109B40007091D4048091D5049091D60420E031E046
:109B500040E050E00E9438568091A2049091A30406
:109B6000820F931F9093A3048093A204DDCA0E94E6
:109B7000BC024CE567ED77E00E943A038091DF0775
:109B800080FF10C08091180390911903875B934068
:109B900038F480911803909119038E5E924010F46E
:109BA0000E94FC1A0E948632A5CCF095E195FF4FE9
:109BB000D3CD20919E0430919F04245130403093A6
:109BC000A1042093A0042C5E3F4F1092880481E0F2
:109BD0008093B7030C94FC4441E00C94F93B96014C
:109BE000D7FC42C0359527953093A5042093A40453
:109BF0009B0177FD36C0359527953093A3042093BC
:109C0000A20425C98091D807A82FB0E0AA0FBB1FD6
:109C1000FD01EB55F84F0190F081E02DF7FD34C0C8
:109C2000E734F10514F40C94343C0C94D83B299A95
:109C30000C94BA3B81E08093CC0497CE81E0809372
:109C4000CA0437CE299ADBCB909581959F4F0C940F
:109C50003C3C81E08093C90467CA81E08093CB04D7
:109C6000E4C92F5F3F4FC7CF2F5F3F4FBBCFF0956A
:109C7000E195FF4FE5C821503F4FF5CB81509F4FF5
:109C8000D5CB21503F4F16CCF095E195FF4FC8CF73
:109C900060926908AE960FB6F894DEBF0FBECDBFD6
:109CA000DF91CF911F910F91FF90EF90DF90CF90B8
:109CB000BF90AF909F908F907F906F905F904F90EC
:109CC0003F902F9008958091280590912905A091AB
:109CD0002A05B0912B058093300590933105A09310
:109CE0003205B093330580912C0590912D05A091FC
:109CF0002E05B0912F058093340590933505A093E0
:109D00003605B0933705089510922105109220056D
:109D10001092230510922205089584B1806A84B9B7
:109D20003D9A82E58CBD1DBC459A81E080938908EF
:109D30008AEA80938D0883E880938E088AE0809376
:109D40008F08109291081092900810929308109228
:109D500092081092AF081092B00888E48093B1087E
:109D60008FE08093B20885E08093B3080895EF9266
:109D7000FF920F931F93F894E090EB07FF24EE0CF3
:109D8000FF1CEE0CFF1C0027F7FC0095102F6091C4
:109D90004504709146048091470490914804A801BD
:109DA00097010E9438563093910820939008609153
:109DB0004D0470914E0480914F0490915004A8017D
:109DC00097010E943856309393082093920860912F
:109DD0007E0870917F0880918008909181082AE028
:109DE00030E040E050E00E94C4552091B303309130
:109DF000B4034091B5035091B6030E943856309396
:109E0000990820939808E0913D04F0913E048091D8
:109E10005F0890916008BF010E940356CB01880F34
:109E2000991F860F971F9C01220F331F96FD22C199
:109E30003595279535952795309395082093940867
:109E400080917A0890917B08BF010E940356CB0154
:109E5000880F991F860F971F9C01220F331F96FDB5
:109E600006C135952795359527953093970820930A
:109E7000960810923E0410923D04109260081092D1
:109E80005F0810927B0810927A0880918F088C30BE
:109E900009F484C18D3008F465C08D3009F414C113
:109EA0008E3009F4FCC078948091AF08882309F4BF
:109EB000D5C02091B5083091B608C90181509E4F98
:109EC0008F5F934058F44091B7085091B808CA0189
:109ED00081509E4F8F5F934008F4D4C08091BB089F
:109EE0009091BC0821E08936920724F49093820473
:109EF000809381048091810490918204845E9D4FBF
:109F00002091830430918404821B930B68E671E0F6
:109F10000E940356845B904090938604809385044E
:109F20002091BF083091C0088091E5039091E6032D
:109F30008217930728F480919A06882309F49DC01C
:109F40008091B408873609F04EC18091C108809392
:109F5000E8088091C2088093EA088091C308809342
:109F6000E90841C18A3009F4E0C08B3009F09BCF89
:109F7000E091D907F0E0EE0FFF1FEB55F84F01908D
:109F8000F081E02D2FEFE138F20714F4E1E8FFEF64
:109F9000E038F10514F0EFE7F0E0E093A008E0917D
:109FA000DA07F0E0EE0FFF1FEB55F84F0190F0815C
:109FB000E02D4FEFE138F40714F4E1E8FFEFE0386B
:109FC000F10514F0EFE7F0E0E093A108E091D80785
:109FD000F0E0EE0FFF1FEB55F84F0190F081E02D00
:109FE0006FEFE138F60714F4E1E8FFEFE038F10530
:109FF00014F0EFE7F0E0E093A208E091D707F0E07B
:10A00000EE0FFF1FEB55F84F0190F081E02D8FEF21
:10A01000E138F80714F4E1E8FFEFE038F10514F057
:10A02000EFE7F0E0E093A30880918C048093A4080C
:10A0300080918E048093A508809190048093A60857
:10A04000809192048093A708809194048093A8083B
:10A0500078948091AF08882309F02BCF10922105C6
:10A06000109220051092230510922205BCC02D5F8E
:10A070003F4FF7CE2D5F3F4FDBCE3093E60320936B
:10A08000E5035ECF8091DF0785FF28CF3093210560
:10A090002093200550932305409322051FCF8091E4
:10A0A000B0088093A0088091B1088093A1088091A6
:10A0B000B2088093A2088091B3088093A30880918E
:10A0C00000018093A408EFCE809111088093A0082E
:10A0D000809112088093A108809113088093A208B0
:10A0E000809114088093A308809115088093A40898
:10A0F000809119088093A50880911A088093A6087A
:10A1000080911B088093A70880911E088093A8085F
:10A1100080911C088093A90880911D088093AA084B
:10A1200080911F088093AB08BECE8091AC048093D1
:10A13000A0088091AD048093A1088091AE04809323
:10A14000A2088091AF048093A3088091B00480930B
:10A15000A4088091B1048093A5088091B2048093F3
:10A16000A6088091B3048093A7088091C0048093CF
:10A17000A808837F8093C00480910E0390910F0301
:10A180008093A9088091F0078093AA08A2E0B0E02C
:10A190000E945356802D8093AB0885CE80919A06FD
:10A1A0008630F0F010929A0685E08093A0088091A6
:10A1B0009E0490919F049093A3088093A20880919D
:10A1C00020088093A108809116088093A4088091AC
:10A1D00017088093A508809118088093A60863CE7D
:10A1E0008093A008E4CF1F910F91FF90EF90089506
:10A1F00080918908882309F43BC045988DE898E050
:10A2000090938B0880938A0890913805E92FF0E0AD
:10A21000E854FC4F808180938F089F5F90933805AE
:10A22000963010F010923805109289080E94B74EAF
:10A2300081E080938C080000000000000000000016
:10A24000000000000000000000000000000000000E
:10A2500000000000000000000000000000000000FE
:10A2600000000000000080918D088093AC088EBD36
:10A27000089580918908882311F40DB407FE08958C
:10A2800084E08093E703459A9EB580913A0581303A
:10A2900009F43AC0813008F040C01092AE089093A3
:10A2A0003905913809F45EC020918C08203208F0FD
:10A2B00030C04598000000000000000000000000D1
:10A2C000000000000000000000000000000000008E
:10A2D000000000000000000000000000000000007E
:10A2E00000000000E0918A08F0918B08E20FF11D58
:10A2F00080818EBD80819091AC08890F8093AC08DD
:10A300002F5F20938C080895953519F110923A0526
:10A31000CBCF81E080938908F3CF823009F0C4CF9E
:10A320008091AE08E82FF0E0E253F74F90838F5F03
:10A330008093AE088A3138F0809139059817B1F0D2
:10A340001092AF08E3CF80913905890F80933905CA
:10A35000ABCF809139058B5A8093390582E0809389
:10A360003A05A2CF81E080933A059ECFA4EBB8E0F6
:10A37000EEECF8E08AE101900D928150E1F781E086
:10A380008093AF08C3CF87B18C6087B94298439858
:10A3900010923F0580E88093BE03109240058093A1
:10A3A000BF030895809141058150809341058F3FFF
:10A3B00009F0089584E08093410580918804882302
:10A3C00009F446C0809142088B3508F443C0883CAC
:10A3D00008F040C080913F05815080933F058F3F3A
:10A3E00009F043C080916108815080933F058091BE
:10A3F000BE03813009F48CC086958093BE038091A2
:10A40000BE039091F507892309F457C0429A8091C1
:10A4100010088B3F70F58091400581508093400576
:10A420008F3F39F680917508815080934005809167
:10A43000BF03813009F450C086958093BF0380919B
:10A44000BF0390910F08892309F040C043980895F5
:10A45000809142088436B8F08739C0F280913F0578
:10A46000815080933F058F3FD9F1809110088B3F39
:10A4700090F280917508873E10F180910F08882333
:10A480002CF14398089580913F05815080933F05BA
:10A490008F3F59F780916108815080933F058091EB
:10A4A000BE038130A9F086958093BE038091BE03E0
:10A4B0009091F607892309F0A9CF4298D6CF8A3028
:10A4C00008F0A9CF80910F0887FDDBCF439A08954C
:10A4D00080E88093BE03EACF80E88093BF03AFCFCC
:10A4E00080916108815080933F058091BE03813047
:10A4F00059F086958093BE038091BE039091F70733
:10A500008923D9F2429A83CF80E88093BE03F4CFA7
:10A5100080E88093BE0373CF8091C9008F778093CA
:10A52000C9008091C9008F7B8093C9008091C900C8
:10A530008F7D8093C9005A9A52981092CD0084E181
:10A540008093CC008091C80082608093C80080E135
:10A550008093C9008091CA008F778093CA00809150
:10A56000CA008F7B8093CA008091CA008F7D809340
:10A57000CA008091CA008F7E8093CA008091CA0071
:10A58000877F8093CA008091C9008B7F8093C90028
:10A590008091CA0084608093CA008091CA00826062
:10A5A0008093CA008091C80087FF06C08091CE00CA
:10A5B0008091C80087FDFACF8091C90080688093A0
:10A5C000C90008951F920F920FB60F9211240F9396
:10A5D0001F932F933F934F935F936F937F938F932B
:10A5E0009F93AF93BF93CF93DF93EF93FF9310911C
:10A5F000CE008091C0039091C103019709F44DC032
:10A6000080914205909143050E948E1220914A0547
:10A6100030914B052115310519F12130310509F42F
:10A62000EAC02230310509F4F9C02330310509F4BC
:10A630005DC081E090E09093C1038093C0031092CD
:10A64000490510924805109245051092440587E08F
:10A6500090E00E948512909343058093420522C1A9
:10A660008823A1F5C0914805D0914905609778F3FA
:10A670008091440590914505892B11F4109279033E
:10A680001092490510924805109245051092440514
:10A6900010924B0510924A05DACF1092C103109226
:10A6A000C00387E090E00E94851290934305809359
:10A6B0004205109249051092480510924B051092E0
:10A6C0004A051092470510924605ECC081E090E0E3
:10A6D00090934B0580934A05C0914805D091490558
:10A6E0002196D0934905C0934805C0CF882309F02F
:10A6F000A0CF82E090E090934B0580934A05C091F3
:10A700004805D09149052196D0934905C093480545
:10A710002091460530914705F901F695E795F695A4
:10A72000E795EF70F0703196EB30F10508F09ECFB1
:10A73000812F90E0322F2227822B932B9370805011
:10A74000924063E070E00E9403568F01000F111FDA
:10A75000F801EB55F84F808191819B01281B390B43
:10A76000C90137FD9BC0069754F480919404883C3E
:10A7700008F08DC080919404865F80939404F80162
:10A78000EB55F84F808191819C01220F331F280FD8
:10A79000391F260F371F37FD7EC035952795359514
:10A7A0002795CB010196821793070CF067C02150C3
:10A7B000304080919404843B08F45AC0F801EB5572
:10A7C000F84F80819181A901481B590BCA0163E0B0
:10A7D00070E00E940356CB01880F991F860F971FC8
:10A7E000F801E554F84F918380830B55184FF80119
:10A7F000318320833BCF882309F013CF82E090E0A0
:10A8000090934B0580934A05C0914805D091490526
:10A810002196D0934905C093480528CF882309F095
:10A8200004CF812F90E090934705809346052091B7
:10A830004805309149052230310569F083E090E008
:10A8400090934B0580934A05E9012196D0934905E1
:10A85000C09348050BCF109245051092440517FF91
:10A86000EDCF81E090E09093450580934405E6CFDD
:10A87000F801E554F84F11821082B7CF6150704053
:10A88000261737070CF095CF2F5F3F4F92CF88ECFC
:10A890008093940474CF2D5F3F4F7FCF9095819527
:10A8A0009F4F61CFFF91EF91DF91CF91BF91AF911A
:10A8B0009F918F917F916F915F914F913F912F91D8
:10A8C0001F910F910F900FBE0F901F901895FC01D4
:10A8D0004150504030F001900616D1F73197CF012A
:10A8E00008958827992708955058BB27AA270ED086
:10A8F00011C102D130F007D120F031F49F3F11F4A3
:10A900001EF4F7C00EF4E095E7FBEDC0E92F13D17C
:10A9100080F3BA17620773078407950718F071F47C
:10A920009EF52BC10EF4E0950B2EBA2FA02D0B0136
:10A93000B90190010C01CA01A0011124FF27591B84
:10A9400099F0593F50F4503E68F11A16F040A22F8A
:10A95000232F342F4427585FF3CF469537952795FB
:10A96000A795F0405395C9F77EF41F16BA0B620BFA
:10A97000730B840BBAF09150A1F0FF0FBB1F661F41
:10A98000771F881FC2F70EC0BA0F621F731F841F84
:10A9900048F4879577956795B795F7959E3F08F0AA
:10A9A000B3CF9395880F08F09927EE0F9795879569
:10A9B000089504D06894B111E1C00895C4D088F01E
:10A9C0009F5790F0B92F9927B751A0F0D1F0660F9B
:10A9D000771F881F991F1AF0BA95C9F712C0B130B6
:10A9E00081F0CBD0B1E00895C8C0672F782F8827B9
:10A9F000B85F39F0B93FCCF3869577956795B395F5
:10AA0000D9F73EF490958095709561957F4F8F4F63
:10AA10009F4F0895E89409C097FB3EF49095809568
:10AA2000709561957F4F8F4F9F4F9923A9F0F92F14
:10AA300096E9BB279395F695879577956795B79592
:10AA4000F111F8CFFAF4BB0F11F460FF1BC06F5F78
:10AA50007F4F8F4F9F4F16C0882311F096E911C08A
:10AA6000772321F09EE8872F762F05C0662371F0AB
:10AA700096E8862F70E060E02AF09A95660F771FBF
:10AA8000881FDAF7880F9695879597F9089507D06C
:10AA900008F481E0089503D008F48FEF0895990F2A
:10AAA0000008550FAA0BE0E8FEEF16161706E80798
:10AAB000F907C0F012161306E407F50798F0621BB9
:10AAC000730B840B950B39F40A2661F0232B242B8E
:10AAD000252B21F408950A2609F4A140A6958FEFAD
:10AAE000811D811D089597F99F6780E870E060E0FF
:10AAF00008959FEF80EC089500240A941616170617
:10AB000018060906089500240A941216130614065E
:10AB100005060895092E0394000C11F4882352F0C1
:10AB2000BB0F40F4BF2B11F460FF04C06F5F7F4F79
:10AB30008F4F9F4F089557FD9058440F551F59F060
:10AB40005F3F71F04795880F97FB991F61F09F3F1A
:10AB500079F087950895121613061406551FF2CF43
:10AB60004695F1DF08C0161617061806991FF1CF93
:10AB700086957105610508940895E894BB276627BA
:10AB80007727CB0197F90895629FD001739FF00159
:10AB9000829FE00DF11D649FE00DF11D929FF00D6D
:10ABA000839FF00D749FF00D659FF00D9927729FA4
:10ABB000B00DE11DF91F639FB00DE11DF91FBD012F
:10ABC000CF0111240895991B79E004C0991F9617AD
:10ABD00008F0961B881F7A95C9F780950895AA1BDF
:10ABE000BB1B51E107C0AA1FBB1FA617B70710F078
:10ABF000A61BB70B881F991F5A95A9F780959095AA
:10AC0000BC01CD01089597FB092E07260AD077FDD8
:10AC100004D0E5DF06D000201AF4709561957F4FCF
:10AC20000895F6F7909581959F4F0895A1E21A2E09
:10AC3000AA1BBB1BFD010DC0AA1FBB1FEE1FFF1FE0
:10AC4000A217B307E407F50720F0A21BB30BE40B30
:10AC5000F50B661F771F881F991F1A9469F7609577
:10AC60007095809590959B01AC01BD01CF01089531
:10AC700097FB092E05260ED057FD04D0D7DF0AD04A
:10AC8000001C38F450954095309521953F4F4F4F1B
:10AC90005F4F0895F6F790958095709561957F4F79
:10ACA0008F4F9F4F0895F999FECFB2BDA1BDF89A7D
:10ACB000119600B40895F999FECFB2BDA1BD00BCB4
:10ACC00011960FB6F894FA9AF99A0FBE089501906A
:0AACD000F2DF1A94E1F70895FFCFB8
:10ACDA000A010101FF6401C800416E676C654E6993
:10ACEA00636B20202020202020416E676C65526F04
:10ACFA006C6C202020202020204163634E69636B06
:10AD0A00202020202020202020416363526F6C6C79
:10AD1A002020202020202020204779726F47696553
:10AD2A00722020202020202020486967687420563D
:10AD3A00616C756520202020204163635A20202001
:10AD4A00202020202020202020476173202020203E
:10AD5A00202020202020202020436F6D70617373F3
:10AD6A002056616C7565202020566F6C746167658A
:10AD7A00202020202020202020456D7066616E67EB
:10AD8A002020202020202020204779726F204B6F1E
:10AD9A006D70617373202020204D6F746F7220468E
:10ADAA00726F6E7420202020204D6F746F722052B3
:10ADBA006561722020202020204D6F746F72204C14
:10ADCA006566742020202020204D6F746F722052F7
:10ADDA00696768742020202020202020202020203D
:10ADEA002020202020202020202020202020202059
:10ADFA002020202020202020202020202020202049
:10AE0A002020202020202020204D4B334D61672018
:10AE1A0043616C537461746520536572766F2020A8
:10AE2A002020202020202020202020202020202018
:10AE3A002020202020202020202020202020202008
:10AE4A0020202020202020202020202020202020F8
:10AE5A0020202020202020202020202020202020E8
:10AE6A0020202020202020202020202020202020D8
:10AE7A0020202020202020202020202020202020C8
:10AE8A002020202020202020204B616C6D616E5FE5
:10AE9A004D61784472696674202020202020202089
:10AEAA002020202020202020202020202020202098
:10AEBA002020202020202020204750535F4E696305
:10AECA006B20202020202020204750535F526F6C97
:10AEDA006C2020202020202020FFFFFC010164009C
:10AEEA00C409C409007D0000FF03737373010102E2
:10AEFA00030405060708090A48616C6C6F20576548
:10AF0A006C74000000000000000000000000000057
:10AF1A000000000000000000000000000000000027
:10AF2A000000000000000000000000000000000017
:10AF3A000000000000000000000000000000000007
:10AF4A0000000000000000000B01426567696E6E98
:10AF5A00657200004E6F726D616C000053706F7203
:10AF6A007400006400F40190D0030090D00300380C
:10AF7A000130FB103A40089696020A64465A41404C
:10AF8A0064ECFF0B050000640A0B0D0B0C0E0101AB
:02AF9A000100B4
:00000001FF
